:02000004000FEB
:1010000040C90020DD130F00E5130F00E7130F00A8
:10101000E9130F00EB130F00ED130F0000000000A9
:10102000000000000000000000000000C9130F00D5
:10103000F1130F0000000000F3130F00F5130F0071
:10104000F7130F00F7130F00F7130F00F7130F003C
:10105000F7130F00F7130F00F7130F00F7130F002C
:10106000F7130F00F7130F00F7130F00F7130F001C
:10107000F7130F00F7130F00F7130F00F7130F000C
:10108000C12C0F00712A0F00F7130F00F7130F0088
:10109000F7130F00F7130F00E12A0F00F7130F00EB
:1010A000F7130F00F7130F00F7130F00F7130F00DC
:1010B000F7130F00F7130F000000000000000000FE
:1010C000F7130F00F7130F00F7130F00F7130F00BC
:1010D000F7130F00F7130F00F7130F00F7130F00AC
:1010E000F7130F00F7130F00C5150F0000000000E5
:1010F00000000000F7130F0000000000F7130F00BE
:1011000000000000000000000000000000000000DF
:1011100000000000000000000000000000000000CF
:1011200000000000000000000000000000000000BF
:1011300000000000000000000000000000000000AF
:10114000000000000000000000000000000000009F
:10115000000000000000000000000000000000008F
:10116000000000000000000000000000000000007F
:10117000000000000000000000000000000000006F
:10118000000000000000000000000000000000005F
:10119000000000000000000000000000000000004F
:1011A000000000000000000000000000000000003F
:1011B000000000000000000000000000000000002F
:1011C000000000000000000000000000000000001F
:1011D000000000000000000000000000000000000F
:1011E00000000000000000000000000000000000FF
:1011F00000000000000000000000000000000000EF
:10120000DFF80CD000F0A0F900480047E9540F00C7
:1012100040C9002080F308888E46104730B450E85B
:10122000012F93B2C48923448489A34228BF1B1B86
:101230000489A34202BFBFF32F8F002007E0C3EA57
:10124000020340E80134002CE9D14FF001000A60AC
:1012500030BC704750E8012FC2EA024240E8012149
:101260000029F7D1704730B450E8022F1FFAA2F3DB
:10127000C488A34202BFBFF32F8F00200DE0C489B2
:1012800023448489A34228BF1B1BC2EA034340E8CE
:101290000234002CE8D14FF001000A6030BC7047E6
:1012A00050E8022FC2EA224240E802210029F7D189
:1012B0007047034653E8022FD988B2EB324F4FF004
:1012C000000017BF92B241EA014142EA014104E045
:1012D0005A68B2EB324F08BF012043E80212002ADD
:1012E000E8D1704730B4044654E8000F0D4644E896
:1012F0000053002BF8D1156030BC704730B4044661
:1013000054E8000F40EA010544E80053002BF7D1F0
:10131000156030BC704730B4044654E8000F00EA52
:10132000010544E80053002BF7D1156030BC70472D
:1013300030B4044654E8000F80EA010544E8005345
:10134000002BF7D1156030BC704730B4044654E828
:10135000000F00EB010544E80053002BF7D11560A6
:1013600030BC704730B4044654E8000FA0EB0105D0
:1013700044E80053002BF7D1156030BC704770B4BF
:1013800004464FF0000054E8006F0D68AE4207BFFE
:1013900044E80023012044E800630E60002B1CBFDA
:1013A0000020F0E770BC704730B4044654E8000FEA
:1013B00088422CBF451A054644E80053002BF5D15E
:1013C000156030BC704700001EF0040F0CBFEFF337
:1013D0000880EFF3098007F001BF0000064880474E
:1013E00006480047FEE7FEE7FEE7FEE7FEE7FEE70A
:1013F000FEE7FEE7FEE7FEE7E52A0F0001120F0019
:101400002DE9F05F0546002092469B468846064639
:10141000814640241BE0284641464746224600F0CC
:1014200083F853465A46C01A914110D311461846C4
:10143000224600F016F82D1A67EB01084F462246A7
:101440000120002100F00DF817EB00094E41201E8D
:10145000A4F10104DFDC484631462A464346BDE894
:10146000F09F202A04DB203A00FA02F100207047A6
:101470009140C2F1200320FA03F3194390407047D2
:101480000048704784BE0F0010B5441A03469442CA
:1014900009D28418114403E011F8013D04F8013D1C
:1014A000521EF9D210BD40EA0104A40703D009E09E
:1014B00010C9121F10C3042AFAD203E011F8014B1D
:1014C00003F8014B521EF9D210BDD2B201E000F870
:1014D000012B491EFBD270470022F6E710B51346D8
:1014E0000A4604461946FFF7F0FF204610BD421C8D
:1014F00010F8011B0029FBD1801A704730B5044653
:101500000020034600E05B1C934203D2E05CCD5C0C
:10151000401BF8D030BD034611F8012B00F8012B19
:10152000002AF9D118467047202A04DB203A21FA14
:1015300002F00021704721FA02F3D040C2F12002EC
:101540009140084319467047064C074D06E0E06895
:1015500040F0010394E8070098471034AC42F6D3FA
:10156000FFF752FE88CE0F00A8CE0F0070B58C1882
:1015700010F8015B15F0070301D110F8013B2A11A7
:1015800006D110F8012B03E010F8016B01F8016B94
:101590005B1EF9D12B0705D40023521E0DD401F890
:1015A000013BFAE710F8013BCB1A921C03E013F859
:1015B000015B01F8015B521EF9D5A142D8D300208E
:1015C00070BD0000054B4FF0FF321A6053F8042C39
:1015D000034B1A601A68034B1A60704704BA025032
:1015E0003CA9002008BA025001EB820204388A426A
:1015F00001D10020704752F8043D1BBA40F8043F67
:10160000F5E7000000B5374B8FB019461A68009215
:10161000009AD207FAD5344B344A1A600A6801920C
:10162000019AD007FAD5324A1A600A680292029AE1
:10163000D207FAD52F4A1A600A680392039AD00794
:10164000FAD52D4A1A600A680492049AD207FAD58C
:101650002A4A1A600A680592059AD007FAD5284ADC
:101660001A600A680692069AD207FAD5254A1A60C5
:101670000A680792079AD007FAD5234A1A600A68BF
:101680000892089AD207FAD5204A1A600A68099285
:10169000099AD007FAD51E4A1A600A680A920A9A6D
:1016A000D207FAD51B4A1A6008680B900B98C0073E
:1016B000FAD51A600A680C920C9AD007FAD5164A25
:1016C0001A600A680D920D9AD207FAD5134A1A6069
:1016D0000E210D230F22002000F088FD0FB05DF8D1
:1016E00004FB00BFB0B0025080B00250804301291B
:1016F00040633921807001298020542100D1349029
:10170000C0403490C0302029C0530D900041389023
:10171000832308C880E3102100413821CF4308C843
:1017200010B5504B96B01C461A680192019AD20728
:10173000FAD54D4B4D4A1A6022680292029AD2079E
:10174000FAD54B4A1A604B4A42EA8040226803921B
:10175000039AD207FAD5186022680492049AD00737
:10176000FAD5454A1A60A2F5800242EA8141226810
:101770000592059AD207FAD5196022680692069A50
:10178000D007FAD53D4A1A6022680792079AD10716
:10179000FAD53B4A1A6022680892089AD207FAD50D
:1017A000384A1A6022680992099AD007FAD5364A4F
:1017B0001A6022680A920A9AD107FAD5334A1A6047
:1017C00022680B920B9AD207FAD5314A1A60226826
:1017D0000C920C9AD007FAD52E4A1A6022680D9204
:1017E0000D9AD107FAD52C4A1A6022680E920E9AE9
:1017F000D207FAD5294A1A6022680F920F9AD007A9
:10180000FAD5274A1A60216810911099C907FAD5AC
:101810001A60144B1A46196811911199C807FAD524
:10182000114B20491960116812911299C907FAD514
:101830001D491960116813911399CC07FAD50B490A
:101840001960116814911499C807FAD517491960DD
:10185000116815911599C907FAD5154A1A6016B07D
:1018600010BD00BFB0B0025080B0025040044190A3
:1018700000862929D81001C840144190401421291C
:10188000401465210034409000310C90C0400C9011
:10189000C030202940960D9000416090031645C845
:1018A0000086112100416021594644C840144590EA
:1018B00040142D90F0B5464B89B01D461C6801942C
:1018C000019CE407FAD5434BDFF810C1DFF810E1C3
:1018D00013449B000A181B681E2A88BFC0F11E0112
:1018E0001F330A185B095A43B2F5806F88BF4FF463
:1018F00080614FF0000484BFB1FBF3F1091A00F1DD
:10190000A05000F52C402746A14233DC2A680492FF
:10191000049AD207FAD5304A1268296805910599C8
:10192000CF07FAD52D482E4C0260002216469A4267
:1019300002F1010140D12A4C134621F00101002699
:101940008B423CD32B680693069BDE07FAD5254BCA
:101950001B682C680794079CE407FAD503600023F2
:101960001F481C469A422DD11D4A00208B422CD381
:1019700009B0F0BD2A680292029AD207FAD502197C
:10198000920012682E680396039EF607FAD5CCF8EB
:10199000002000229A4202F1010206D11E4622F0E6
:1019A0000102964204D30134AEE7CEF80070F1E7AD
:1019B000CEF800700136F4E726600A46B7E72660E5
:1019C0000133BDE704600133CCE710600133CDE79C
:1019D000B4B0025024AC00147CB00250D4B0025019
:1019E000D8B0025078B00250F0B5294D85B02C46E1
:1019F0002E680096009EF607FAD500F1A05000F57B
:101A00002C4080000568206801900198C707FAD52E
:101A10002048214F056002EB8306B24229D15A1CAF
:101A20001D4E22F001020027934227D32368029320
:101A3000029BDE07FAD5194B0B449B001B681F3332
:101A40005B099A4213D2216803910399C907FAD519
:101A5000154400219B1A104A05600846994210D38C
:101A60005A1C0D4922F00102002093420CD305B00C
:101A7000F0BD52F804EBC7F800E0CEE73760013361
:101A8000D2E710600131E9E708600133EDE700BFFC
:101A9000B4B00250D4B00250D8B0025024AC0014FC
:101AA00010B5494B94B019461A680092009AD207B3
:101AB000FAD5464B464A1A600A680192019AD40741
:101AC000FAD5444A1A600A680292029AD007FAD5F7
:101AD000414818600A680392039AD207FAD53F4A30
:101AE0001A600A680492049AD407FAD53C4A1A602C
:101AF0000A680592059AD207FAD53A4A1A600A6826
:101B00000692069AD407FAD5374A1A600A680792ED
:101B1000079AD207FAD5354A1A600A680892089AD5
:101B2000D407FAD5324A1A600A680992099AD2078C
:101B3000FAD5304A1A600A680A920A9AD407FAD586
:101B40002D4A1A600A680B920B9AD207FAD52B4AD3
:101B50001A600A680C920C9AD407FAD5284A1A60BF
:101B60000A680D920D9AD207FAD5264A1A600A68B9
:101B70000E920E9AD407FAD5234A1A600A680F9279
:101B80000F9AD207FAD5214A1A600F4B19461C68E2
:101B90001094109CE407FAD50C4B1860086811905B
:101BA0001198C407FAD51A600A681292129AD007DF
:101BB000FAD5174A1A600A681392139AD207FAD50F
:101BC000144A1A6014B010BDB0B0025080B0025078
:101BD0008090652100040990409665908080612185
:101BE00080200821802064900081619000461021AF
:101BF000008111210041442180202029024610C883
:101C000000860921802060214021282940966521F5
:101C100040962529594614C810B5544B98B019461A
:101C20001A680192019AD207FAD5514B514A1A60AB
:101C30000A680292029AD407FAD54F4A1A600A68D3
:101C40000392039AD007FAD54C4818600A680492A8
:101C5000049AD207FAD54A4A1A600A680592059A88
:101C6000D407FAD5474A1A600A680692069AD2073C
:101C7000FAD5454A1A600A680792079AD407FAD536
:101C8000424A1A600A680892089AD207FAD5404A6E
:101C90001A600A680992099AD407FAD53D4A1A606F
:101CA0000A680A920A9AD207FAD53B4A1A600A6869
:101CB0000B920B9AD407FAD5384A1A600A680C922C
:101CC0000C9AD207FAD5364A1A600A680D920D9A14
:101CD000D407FAD5334A1A600A680E920E9AD207D0
:101CE000FAD5314A1A600A680F920F9AD407FAD5CA
:101CF0002E4A1A600A681092109AD207FAD52C4A16
:101D00001A601A4B19461C681194119CE407FAD505
:101D1000174B1860086812901298C407FAD51A6019
:101D20000A681392139AD007FAD5124A1A600A6801
:101D30001492149AD207FAD51E4A1A600A681592AC
:101D4000159AD407FAD51C4A1A600A681692169A90
:101D5000D007FAD5194A1A600A681792179AD2075B
:101D6000FAD5174A1A6018B010BD00BFB0B00250C3
:101D700080B0025000936521000431904096659038
:101D80000083612100C3302100C364900081619011
:101D900000461021008111210041442100C3202967
:101DA0000C4610C80086312100C3602140C128299B
:101DB000409665210013319040962529594614C854
:101DC000400432492DE9F041814B1D689868203369
:101DD000A0B01E461A680192019AD707FAD57D4B2A
:101DE0007D4A1A6032680292029AD407FAD57B4A79
:101DF0001A607B4A1446116803910399C907FAD502
:101E0000784A1168C1F3402137680497049FFF079F
:101E1000FAD5754F1F6027680597059FFF07FAD50C
:101E20001768002900F0CF80B90540F1CC803168F7
:101E300006910699CF07FAD56C4919602168079178
:101E40000799C907FAD51168C1F340213768089787
:101E5000089FFF07FAD5664F1F6027680997099FFB
:101E6000FF07FAD51268002900F0AF80910540F114
:101E7000AC8032680A920A9AD207FAD5564A1A609A
:101E800032680B920B9AD707FAD55A4A1A60316812
:101E90000C910C99CC07FAD55749196031680D910E
:101EA0000D99C907FAD55549196031680E910E99F7
:101EB000CF07FAD55249196031680F910F99CC07B5
:101EC000FAD550491960504B1E4619681091109967
:101ED000C907FAD53F4C4D4B236033681193119BD2
:101EE000DB07FAD54A4B236033681293129BDF0756
:101EF000FAD5484B23603A4B9846196813911399C9
:101F0000C907FAD5324F386033681493149BDB0746
:101F1000FAD5226033681593159BD807FAD53E4B46
:101F2000236033681693169BD907FAD53B4B236081
:101F300033681793179BDA07FAD5394B2360336858
:101F40001893189BDB07FAD5364B23603368199337
:101F5000199BD807FAD5344B236033681A931A9B20
:101F6000D907FAD5314B236033681B931B9BDA07E3
:101F7000FAD52F4B236000F0D3F908BBD8F8003016
:101F80001C931C9BDB07F9D53D6033681D931D9B9B
:101F9000D907FAD5274B236033681E931E9BDA07B7
:101FA000FAD5254B2360D8F800301F931F9BDB0721
:101FB000F9D50C4B1B6813F4805F204B08BF184603
:101FC00020B0BDE8F0811E48FAE71E48F8E700BFE0
:101FD00090B0025080B0025000100251C01F722910
:101FE000B4B0025088B00250C0CF0129C01F0E29E2
:101FF000C03F002940010249003184A80000164971
:10200000400108A180440888B0B00250C0447088E4
:1020100080077A41C0077E4100006A498006164960
:1020200040006E49000200210082202140822021D0
:102030008082242140A161A100C861510308F10000
:102040000108F1000208F10008B540B1202801465E
:102050004FF0070228BF20210020FFF72BFC024B86
:1020600000221A6008BD00BF1CB802507FB51C6872
:102070001CB901F01F041F2C27D1174C25462668D8
:102080000196019EF607FAD500F1A05000F52C400C
:10209000800000682C680394039CE407FAD50F4C79
:1020A00000EB611020600E4801F01F0400680290F0
:1020B0001F2C18BFC94302980FBF106001F01F0109
:1020C00000FA01F111600021196010684300C00F8F
:1020D000136004B070BD00BFB4B00250E4B0025051
:1020E000DCB0025030B51E4B85B01A46196800911D
:1020F0000099CC07FAD500F1A05000F52C408000E3
:10210000016813680193019BD807FAD5154B164C4B
:102110001868164D1F30202390FBF3F0013800287B
:1021200010DA00230130400153B1A0F120014FF03B
:102130000042134204D1013881424FEA5202F8D1E1
:1021400005B030BD13680393039BDB07FAD5431832
:1021500023602B680293029B002BE3D10138DEE75A
:10216000B4B00250ACB00250E4B00250DCB0025047
:102170000A460021AFF3008038B5A0F12003B3F583
:10218000426F05462CD88F2826D800F1470300F16E
:102190006604DB064FEA541400D0013464013F3476
:1021A000A409013411B1A1421AD30C46E3004FF443
:1021B0008050B0FBF3F0202828BF202002B110602F
:1021C000084B01221A60214600F068F82846214693
:1021D00000F088F8002038BD00F11F046409DDE735
:1021E000014838BD1CB802502221F00070B52648C5
:1021F00088B0054604680094009CE607FAD5234899
:10220000234C0460234C44EA83432C680194019CD2
:10221000E407FAD50360930143EA824242F0104496
:1022200044F4C0442B680293029BDE07FAD5046095
:102230002B680393039BDB07FAD5174B03608B01D5
:1022400043EA814141F0104343F4C0432E680496B1
:10225000049EF607FAD503602B680593059BDE07FD
:10226000FAD5046041F058412B680693069BDC07C1
:10227000FAD5016042F058422B680793079BDB07B1
:10228000FAD5026008B070BDB0B0025080B0025004
:10229000C0210229807100988061189030B5002219
:1022A0000C4C49001346023840F6FC75904202F18E
:1022B0000102CABF236025605B181E2A04F10404D2
:1022C000F4D1054A19441360044B054A19609A6019
:1022D00030BD00BF00B0025078B002507CB0025058
:1022E00020F80F000C4B18603F3020F03F008901B0
:1022F000403058609960D9601961596199611C3307
:102300000648196082B002680192019AD207FAD594
:10231000196002B0704700BF90B00250B4B00250D4
:102320002DE9F04192B0012303930493624B1D46C3
:102330001A680592059AD207FAD5604C604B236063
:10234000604B19461A680692069AD707FAD55E4B73
:102350001A68D60400F1A8802A680792079AD00765
:10236000FAD55A4A22600A680892089AD207FAD522
:102370001E68C6F30036002E40F098801220FFF74A
:10238000B1FE07461320FFF7ADFE87428CBF122037
:102390001320FFF7A7FE471EFFF734F903AB01AA8E
:1023A00039461220FFF762FE04AB804602AA394686
:1023B0001320FFF75BFE00EB4800022832D0032811
:1023C0003ED0012874D12B680993099BDB07FAD50D
:1023D0003F4B23602B680A930A9BD807FAD53D4BE5
:1023E00023602B680F930F9BD907FAD53A4B2360D4
:1023F0002B681093109BDA07FAD5384B23602B68B3
:102400001193119BDB07FAD5354B2360013F25D58E
:102410001023192218210020FFF7E8FE304612B0E1
:10242000BDE8F0812B680B930B9BD907FAD52D4B98
:1024300023602B680C930C9BDA07FAD52A4BCFE765
:102440002B680D930D9BDB07FAD5284B23602B6877
:102450000E930E9BD807FAD5254BC1E703AB01AA13
:1024600039461220FFF702FE04AB044602AA3946A1
:102470001320FFF7FBFD10EB440402D1FFF7CCFB68
:10248000C4E7FFF70DFB022C08D0032C09D0012C68
:1024900010D117211620FFF743F9B7E715211420B3
:1024A000F9E70F210E20F6E7124EB7E7124EB5E717
:1024B000124EB3E7124EB1E7B0B0025080B00250F6
:1024C00000084A51B4B0025088B0025000084E5182
:1024D00000065A4940065E49000442410014424940
:1024E00040042E49000652494006564900063A4922
:1024F00040063E490608F1000708F1000408F10013
:102500000508F100014B1860704700BF08BA02507F
:10251000014B1860704700BF04BA0250094BC24318
:102520001A60043B82B01B680193074B019A10426A
:1025300004D0064A1060186802B0704720BF1A68BD
:102540000192F3E704BA02503CA9002008BA0250F5
:10255000FEF79ABFFEF7C2BF0A460021FEF7BEBFD4
:102560002DE9F74305460E469946114600F060FAFC
:102570000446002840F08480002E00F08580002969
:1025800000F08480B9F1200F40F0828005F144040E
:10259000082205F104082046FFF726F805F1240774
:1025A000082231464046FFF71FF806F120010822B5
:1025B0003846FFF719F802A94FF4807041F8049DDE
:1025C000FFF7D6FD002865D1334A4FF480731360BE
:1025D000012193600823314AFFF706FA01210846DA
:1025E00005232F4AFFF700FA0823424601211C2049
:1025F000FFF7FAF908233A4601210320FFF7F4F91F
:102600002246082301210220FFF7EEF90823254A7C
:1026100001211A20FFF7E8F90523234A01211B2095
:10262000FFF7E2F90823214A01211420FFF7DCF922
:1026300008231F4A01211520FFF7D6F9082305F1C9
:10264000640201211620FFF7CFF9082305F1840267
:1026500001211720FFF7C8F90823164A01210B2092
:10266000FFF7C2F9FFF7AEFB04460198FFF7ECFC59
:10267000114B002C18BF1C46A4212846FFF76CFF05
:10268000204603B0BDE8F0830C4CF9E70C4CF7E7AB
:102690000C4CF5E7084CEFE790B00250FCCD0F0072
:1026A00074CE0F00BCCD0F0060CE0F0020CE0F0007
:1026B00040CE0F00DCCD0F008408F0007608F0005B
:1026C0008008F0008108F00038B50D460446B0B12E
:1026D000A02200210430FFF73DFF95B129460822D2
:1026E00004F16400FEF780FF082205F1200104F1E7
:1026F0008400FEF779FF044B2360002038BD0348B7
:1027000038BD034838BD00BFDD55AABB7108F000D5
:102710008308F0002DE9F041069F044615461E4649
:10272000FFF7D2FF38B93B46324629462046BDE87E
:10273000F041FFF715BFBDE8F08100002DE9FF4132
:10274000144B04460E460FCB8DE80F00204600F0D8
:102750007FF98046B0B9CEB1636A251D01953BB9BA
:1027600001236362226F04F13001684600F088F8AB
:102770002B46043E243453F8042B12BAA34246F8E5
:10278000042FF8D1404604B0BDE8F081DFF808809E
:10279000F8E700BF8CCD0F000502F00038B5044605
:1027A00068B1051D28467021FFF7D6FE2846202275
:1027B0000449FFF7CDFE044B2360002038BD0348D9
:1027C00038BD00BF9CCD0F00DD55AABB0002F00054
:1027D000294B2DE9F04304460E4615460FCB85B034
:1027E0006F468DE80F002DB94FF00009484605B03F
:1027F000BDE8F083204600F02BF981460028F5D192
:10280000231D0193636AA3BB236F8BB1C3F14008FF
:10281000A84528BFA84604F1300031461844424676
:10282000FFF796FE236F434446442367A5EB080554
:10283000226F402A06D104F13001384600F020F81A
:102840000023236705F03F0835F03F0505D03146EA
:102850002A46384600F014F82E44B8F1000FC3D0D1
:102860004246314604F13000FFF772FEC4F8708032
:10287000BCE7DFF80890B9E78CCD0F000C02F00040
:102880002DE9F74F314B44688046924699461A68C5
:10289000002AFCD12E4B9B461A68002AFCD14FF02F
:1028A000FF300191FFF72EFE8020FFF731FE294D0A
:1028B000294A2A4F2A4E012307202B60A2F59E7237
:1028C000C2F83C011360636A3B60A36A3360D8F8C6
:1028D000003042F8043CD8F8083020469847019967
:1028E000D9F80030002BFBD1BAF1000F20D11D4BDD
:1028F00004221A60D9F80030002BFBD1DBF800A0CD
:10290000BAF1000FFAD1D8F80C30204698473B684E
:1029100063623368A362144BC3F800A0C3F844A1F8
:10292000D9F80030002BFBD12B6003B0BDE8F08F4D
:10293000236A012B04BF0C4A13600C4B4020196022
:10294000C3F804A0FFF7EAFDD4E700BF10B90250B6
:1029500020BC025018B8025000B90250CCB7025047
:10296000D0B70250C8B7025084B6025028BC0250FB
:10297000084B1B681B0EF02B08D1074B1A68074B3E
:102980009A4205D1064B0020186070470520704719
:102990000620704728B9025024BA02500000E020F7
:1029A0000CBA02500C4B1B68C3610C4B1B68836153
:1029B0000B4B1B6843610B4B1B6803610A4B1B6885
:1029C000C3600A4B1B688360094B1B684360094B5B
:1029D0001B680360704700BF5CB6025058B60250D7
:1029E00054B6025050B602504CB6025048B602508F
:1029F00044B6025040B602500C4BC2691A6082695C
:102A000043F8042C426943F8082C026943F80C2C63
:102A1000C26843F8102C826843F8142C426843F8CB
:102A2000182C026843F81C2C704700BF5CB602509B
:102A300030B10268034B04489A4208BF0020704737
:102A400002487047DD55AABB8208F0007108F0000B
:102A500030B10268034B04489A4208BF0020704717
:102A600002487047DD55AABB0202F0000002F000E8
:102A700002490248091F0968006808478058002079
:102A800000F02EB970B50E46144900EB400001EB82
:102A9000C0051446E86A183520B101280FD0022875
:102AA00005D113E0284600F051F9A04201D20024DC
:102AB00011E022463146284600F080F90BE0284616
:102AC00000F044F9A042F4D20446F2E73146284629
:102AD00000F047F90446204670BD0000B49800207D
:102AE00006F08AB930B54FF0805000228300D0F84C
:102AF0003011C3F80C21C3F81021624B1A60624BED
:102B00001B68624C2360604B1B1D1B68241D2360E7
:102B10005D4B08331B68241D23605B4B0C331B6823
:102B2000241D2360584B10331B68241D2360564B13
:102B300014331B68241D2360534B18331B68534CFC
:102B400020342360504B1C331B68241D23604E4BE4
:102B500020331B68241D23604B4B24331B68241D2A
:102B60002360494B28331B68241D2360464B2C33BC
:102B70001B68241D2360444B30331B68434C403496
:102B80002360414B34331B68241D23603E4B383394
:102B90001B68241D23603C4B3C331B68241D2360B1
:102BA000394B40331B68241D23600124082902D1BE
:102BB000D0F8343113B1082904D006E0354B34493C
:102BC000196005E0D0F8343113B1082904D006E0CB
:102BD000314BFB21196005E0D0F8343113B10829DD
:102BE00008D00EE090F858322C48016863F30301D6
:102BF000016002E0D0F834311BB929494FF400706C
:102C0000086028480168C90702D06FF0010101601F
:102C10002548016841F470010160BFF34F8FBFF395
:102C20006F8F4FF01021D1F80002002803DBD1F89C
:102C30000402002822DA1D4B1C601D480468002C89
:102C4000FCD01224C1F800420568002DFCD0C1F868
:102C5000044201680029FCD01A6001680029FCD0F8
:102C6000BFF34F8F10487C380168124A01F4E061CD
:102C700011430160BFF34F8F00BFFDE70F490E48BE
:102C8000086030BD380500400404001020C5004035
:102C9000488103008C56004018F50040E40E0040C7
:102CA000409602400004004088ED00E004E5014049
:102CB00000E401400400FA050090D0030C59002004
:102CC000064808B5002101600068009005F09EFDEF
:102CD00005F06AFB0028FBD108BD0000000101409F
:102CE00010B5124C02202061606111A0A06104F1B6
:102CF0007800E0614FF4805020620020A0626062A2
:102D00000BA1A164E0620D49E1641021A065C4E952
:102D10001410E0650AA1E01DFEF7FDFB09A12046A5
:102D2000FEF7F9FB2020A07110BD0000B498002030
:102D30005465726D696E616C000000002CA9002062
:102D40005254540053454747455200000269C16838
:102D50008A4203D88068401A104400E0501A401E8E
:102D600070472DE9F047C4681746894606464FF07C
:102D700000083069A04201D9051B02E0B168201AA1
:102D80000D1AB0686D1E001BA84200D80546BD4252
:102D900000D33D4670682A4620444946FEF774FB3E
:102DA000B0687F1B2C44A844A944A04200D1002451
:102DB000F460002FDDD14046BDE8F0872DE9F041F9
:102DC00004468846D4E90207C51BE16860681646D8
:102DD0000844B54206D94146FEF756FBB819E060F3
:102DE000BDE8F0812A464146FEF74EFB761B08EB14
:102DF000050132466068FEF747FBE660F0E702E057
:102E000008C8121F08C1002AFAD170477047002075
:102E100001E001C1121F002AFBD1704701212028C7
:102E200003DA81400548014003E0402802DA2038F7
:102E3000814009B10120704700207047FC06FFBDAA
:102E4000800701D00020704701207047406800686B
:102E5000401E084201D10120704700207047C3681E
:102E60008B4206D811440069491E814201D80120D5
:102E7000704700207047000030B585B00D46164CF5
:102E80001621ADF800101ECC0DF1040C8CE81E00CC
:102E9000124C0221012221706270A0700320E070A8
:102EA000217159206071FE20A071694604F109006A
:102EB0007DDF00280ED1BDF800002A46411CE171DB
:102EC00009212172BDF808100844ADF8080001A9D5
:102ED000034872DF05B030BD30BA0F009C6D002092
:102EE0000858002070B58CB006251822294968467C
:102EF000FEF7CAFA284C042628A1208806EB0040D9
:102F000005F0B6FB0020069007900890099010226B
:102F100006A92648FEF7F2FA0028208806EB0040B2
:102F200034D023A105F0A4FB204802268DF81460BC
:102F300010300A90103804250B9001210AA86EDF8A
:102F400040B106F041F90246208821A106EB00407D
:102F500005F092FB012200210BA86FDF40B106F0C3
:102F600033F90246208824A106EB004005F084FBDB
:102F700069462846FFF780FF002805D12A4C2078B3
:102F800074DF0121207873DF0CB070BD27A105F03C
:102F90006FFBEDE740BA0F003059002041647665C1
:102FA00072746973696E672E2E2E0000C06D00204A
:102FB00049524B20466F756E642C2073657474699A
:102FC0006E672075702077686974656C697374002A
:102FD00073645F626C655F6761705F776869746571
:102FE0006C6973745F7365742829207265747572D7
:102FF0006E6564202573000073645F626C655F67B3
:1030000061705F6465766963655F6964656E746944
:10301000746965735F7365742829207265747572AD
:103020006E65642025730000085800204E6F20490B
:10303000524B20666F756E642C2067656E657261F9
:103040006C20646973636F76657279002DE9F05FB7
:10305000DFF894B05C46DBF84890DBF8245003F0CE
:1030600007FA216B214E00EB01086F1A31884FF0EF
:10307000040A0AEB01401EA105F0FAFA216B404652
:103080004944414500D1002708233A4601F0BAFFE0
:1030900007004FF0010806D0318808EB01401BA162
:1030A00005F0E6FA1CE003F0E3F90022294601F0FE
:1030B00035FADBF8282004463188D946A24209D1E6
:1030C0000AEB014018A105F0D3FAC9E90748C9F88D
:1030D000185005E008EB01402346194905F0D3FAE2
:1030E0003846BDE8F09F0000108000206C59002099
:1030F000456E746572206E72665F6466755F61709E
:10310000705F636F6E74696E756500004661696C0F
:10311000656420746F20636F7079206669726D77C3
:103120006172652E0000000053657474696E67203B
:103130006170702061732076616C6964000000002A
:1031400024BF0F0008B5134602460648009301232A
:10315000008803EB00400B4603A105F09CFA06F043
:10316000CFFC00006C590020526563656976656488
:103170002061206661756C74212069643A20307882
:10318000253038782C2070633A2030782530387814
:103190002C20696E666F3A20307825303878000030
:1031A000024605480121008801EB004003A105F01B
:1031B00063FA06F0A5FC00006C59002052656365B7
:1031C0006976656420616E206572726F723A203094
:1031D00078253038782100002DE9F84F254C8146BC
:1031E000924660880E46814241D800274FF6FF780C
:1031F0008DF80070684600F0F5F822786078A188B4
:10320000884201DA401C00E00020C0B2904204D1A4
:103210009DF8000000F032F927E065786078884278
:1032200001DA401C00E0002060709DF8000000F012
:1032300025F9454519D0A068B9F1000F40F835A02F
:103240000DD066B16188E068324605FB0100494651
:10325000FEF71AF9A06800EBC500868002E000EBDB
:10326000C50087800020BDE8F88F0420FBE7092017
:10327000F9E700004458002010B50E4C03E0401C54
:1032800000E00020207020786178814210D0227800
:103290006188E068A36802FB010003EBC20153F8F8
:1032A0003220898890472078A1888842E9DAE6E7C9
:1032B00010BD00004458002030B5CB0008339DB24B
:1032C00093074FF0000401D0072030BD044B9A60F3
:1032D0002A44DA605C701C7058809980002030BDF0
:1032E00044580020014801F03CBB00005C5800201D
:1032F00070B514460E46050004D10B4940F2C510C6
:1033000000F000F93CB12868012EC4600AD0002109
:103310008160002070BD04494FF4E37000F0F2F8C2
:10332000072070BD0121F3E7CCC30F0038B50E486C
:1033300008235822416800910C49006802F080F986
:1033400000280FD10A4A69460A4801F00FFB040021
:1033500008D10121074801F0D8FB064901200839AE
:103360000870204638BD000058BB0F003C85002087
:1033700081A90F005C58002070B516460D46040068
:1033800004D10C4940F2D51000F0BCF80A4885423F
:1033900001D9072070BD0948266101F0E2FA2844EE
:1033A0006060A06800B1A5602146BDE870400020C3
:1033B00008F03EB8CCC30F0017FCFF005C5800209B
:1033C00010B5040004D106494FF4F57000F09AF8E6
:1033D000002021462076BDE81040012008F028B8E2
:1033E000CCC30F0070B5044607F0E4F9012803D000
:1033F00010A11D2000F086F8EFF3108172B61D4A6F
:103400009368012083B990604FF0E020D0F880519C
:10341000194B1D401560C0F88031D0F884315360DD
:103420004217C0F8842100202070002900D162B624
:1034300070BD00002E2E5C2E2E5C2E2E5C2E2E5C7F
:103440002E2E5C636F6D706F6E656E74735C6C694D
:10345000627261726965735C7574696C5C617070CD
:103460005F7574696C5F706C6174666F726D2E63EA
:103470000000000094850020FC06FFBD10B5044646
:1034800007F098F9012803D00DA12B2000F03AF89D
:103490001B498868002811D0002C0FD1EFF3108051
:1034A00072B60B684FF0E022C2F800314B68C2F8E8
:1034B000043100228A60002800D162B610BD0000ED
:1034C0002E2E5C2E2E5C2E2E5C2E2E5C2E2E5C6301
:1034D0006F6D706F6E656E74735C6C696272617231
:1034E0006965735C7574696C5C6170705F75746933
:1034F0006C5F706C6174666F726D2E63000000000B
:10350000948500201CB56A46ADF8000001910021A9
:1035100044F20200FFF716FE1CBD0000F8B51F487C
:103520000146446AC06A8D6CAC2802D1486B0544E0
:10353000241A1B4E0094042730882B4607EB0040CA
:10354000184A19A105F0A7F8224629461548FDF7A3
:10355000D5FFE8B13088234607EB00402A4620A17A
:1035600005F091F804F020FF0028FBD102F096FC52
:103570002146284603F090FB040007D03088012143
:1035800001EB004022A100BF05F072F82046F8BD13
:103590003088002407EB004024A1F5E710800020CC
:1035A0006C59002000100F00566572696679696ECB
:1035B0006720424C3A20416464723A2030782530CA
:1035C00038782C205372633A203078253038782CA4
:1035D000204C656E3A2030782530387800000000A5
:1035E000436F7079696E6720626F6F746C6F61648E
:1035F00065723A205372633A203078253038782C3F
:10360000204C656E3A203078253038780000000074
:103610005265717565737420746F20636F707920C3
:10362000424C206661696C65640000004E6F206248
:103630006F6F746C6F6164657220636F7079206E58
:1036400065656465642C20626F6F746C6F6164657E
:10365000722075706461746520636F6D706C657441
:10366000652E000030B595B0040004D12E4940F21B
:103670002740FFF747FF2D494FF6FF70224648804D
:1036800001208DF812004FF65960ADF8100004A922
:103690000120A8DF002844D1254B0FCB8DE80F0077
:1036A000A11C684662DF00283BD121491C226039F9
:1036B0000BA8FDF7E9FE1F4D142205F1C401A8680F
:1036C0001290A0788DF84A002868139006A8FDF79C
:1036D000DBFE12A8069013A807902088231D06AAD7
:1036E0000BA9AADF00281CD11C2205F1D8010BA8C8
:1036F000FDF7CAFEE8681290A0788DF84A00686865
:103700001390142205F1F40106A8FDF7BDFE12A8DE
:10371000069013A80790208804F10C0306AA0BA9B1
:10372000AADF15B030BD000010C00F0008580020FF
:1037300008BB0F0000BA0F00F0B585B00D460400BD
:1037400004D136494FF4B370FFF7DCFE25B9334995
:1037500040F26710FFF7D6FE14216846FDF7BCFE65
:103760002078032308280BD12D48C188491E89B22F
:10377000C1808288002A49D0002947D1C2802370A5
:103780002178607860228DF800208DF801108DF886
:10379000020063780325012B14D0224802212278ED
:1037A000008801EB004020A104F06DFF60780B2839
:1037B00028D101F02FFB8DF80300002001F032FB2F
:1037C00004251FE0207809281CD2DFE800F01B1B2D
:1037D0001B211B1B051B2100D4E902706D46E91C4F
:1037E000666807F06DFE044629193046C91C07F0CB
:1037F00067FE044429193846C91C07F061FE2044BD
:10380000C01CC5B22946684607F09CF805B0F0BD5B
:10381000D4E90112684607F084F8F1E710C00F0000
:1038200008580020305900204446552072657175B3
:10383000657374202564206661696C65642077690E
:103840007468206572726F723A20307825780000B3
:103850002DE9F0411E4C0027217AC90734D01D49BB
:10386000884231D01C4D04261CA1288806EB00405C
:1038700004F0FEFE6088A0F57F41FF3918D028884B
:103880001EA106EB004004F0F3FEA068132140F0F7
:103890000400A060608876DF002816D11B4CC82782
:1038A0004FF47A48611C404688477F1EFAD101E0F8
:1038B000207874DF05F03CFA070005D1288814A1B0
:1038C00006EB004004F0D4FE3846BDE8F08100006D
:1038D00008580020B0CE0F0030590020536875748E
:1038E00074696E6720646F776E20424C4520747255
:1038F000616E73706F72742E000000004469736310
:103900006F6E6E656374696E672E000010BA0F00EB
:10391000424C45207472616E73706F7274207368CC
:10392000757420646F776E2E00000000F8B52A4C85
:1039300007460020217AC9074DD1284D042628A129
:10394000288806EB004004F093FE2D48E76001F064
:1039500097FF00F053FB00283DD103F0A9FC48B1CC
:10396000288828A106EB004004F082FE2A4803F0D4
:1039700093FC02E00320FFF713FC9DF8000027A151
:1039800020F00F00401C20F0F00010308DF80000F7
:10399000288806EB004004F06BFE28A10722684649
:1039A0007CDF08B927487ADF002814D11A48403054
:1039B000FFF758FE00280ED1FFF794FA00280AD12D
:1039C000A06821A140F00100A060288806EB00401B
:1039D00004F04EFE0020F8BD0858002030590020A9
:1039E000496E697469616C697A696E6720424C45F9
:1039F00020444655207472616E73706F72740000BB
:103A000068CF0F00436F7079696E672070656572CB
:103A10002064617461000000BC6D00205573696E04
:103A2000672064656661756C742061647665727484
:103A30006973696E67206E616D6500004466755438
:103A40006573740016BA0F00424C45204446552059
:103A50007472616E73706F727420696E69746961DB
:103A60006C697A65642E00002DE9FE4FA84E07466A
:103A7000041D018830884FF00408A64D4FF0000A5D
:103A80004FF00109424608EB0040212978D040DC84
:103A9000132976D026DC012974D010295DD0112994
:103AA00076D0122970D115469BA104F0E1FD308833
:103AB000E28805EB0040A2A104F0DEFD3088A28878
:103AC00005EB0040A4A104F0D7FD3088228905EB66
:103AD0000040A7A104F0D0FD3088628905EB0040CA
:103AE000A8A1F0E014297AD01A2979D01F294BD146
:103AF000AAA104F0BDFD211D688875DF040043D034
:103B00003188224609EB0140B0A104F0B5FD204602
:103B10001FE0512970D00EDC22296ED023296FD0EE
:103B200024297DD0502979D103B03946BDE8F04F22
:103B3000B44806F009B95229D7D055293BD05629A7
:103B40006CD1B879002869D11321688876DF002804
:103B500064D0BDE8FE4FFFF723BBABA104F088FDA6
:103B600020886880E96809B101208847A9496888E8
:103B700075DF002852D0328809EB0243024604E088
:103B800080E055E087E003E048E0A3A118469AE012
:103B90004FF6FF706880287A400704D4FFF7A2F937
:103BA00008B1FFF7FDFAE968002937D003B0022019
:103BB000BDE8F04F0847FA88F72A14D29107B1F10F
:103BC000404F0ED0D11F8BB2591ECC1701EB94740D
:103BD00024F00304091B591A891D8CB204E077E014
:103BE00087E0144600E0F7242346974904F04BFD94
:103BF00021466888B5DFAAE751E03BE000E00FE02E
:103C000092A104F035FDCDF800A0CDF804A0B8884D
:103C10000022694690DF2AE0FFF7C2FABDE8FE8F76
:103C20006389E28803B096A1BDE8F04F04F02BBD94
:103C30001446A3A104F01CFD764801AA163842F6EA
:103C40000521806A0190CDF808D06888ADDF08B101
:103C5000FFF7A6FA3088BDF8002004EB0040A2A1CF
:103C600004F00AFD00231A46852168887FDF0028BA
:103C7000D2D1D3E7217900916379A279A3A104F08D
:103C80000AFDCBE7B0A104F0F3FCCDF800A020883A
:103C900069468FDFEBE70021688866DF57E7B87970
:103CA0000028BBD03946574806F00AF80028B5D09E
:103CB00007F10801534805F0AFFB0200AED0318890
:103CC00009EB0140ABA103B0BDE8F04F04F0D4BC58
:103CD000B5A104F0CDFC4B4AA089403A0021D38D18
:103CE000984201D102F11C0100232088121D86DFB9
:103CF0002DE707F08BF808B1FFF752FA318803B0CF
:103D000008EB0140BDE8F04FB1A104F0B1BC0000E8
:103D10003059002008580020526563656976656453
:103D200020424C455F4741505F4556545F434F4EDC
:103D30004E5F504152414D5F555044415445000043
:103D40006D61785F636F6E6E5F696E7465727661C8
:103D50006C3A2025640000006D696E5F636F6E6EC3
:103D60005F696E74657276616C3A202564000000AC
:103D7000736C6176655F6C6174656E63793A20255A
:103D800064000000636F6E6E5F7375705F74696DC1
:103D9000656F75743A202564000000005265636504
:103DA0006976656420424C455F4741505F455654F3
:103DB0005F434F4E4E5F504152414D5F555044411D
:103DC00054455F5245515545535400004661696C56
:103DD00075726520746F2075706461746520636FFF
:103DE0006E6E656374696F6E20706172616D65746B
:103DF000657220726571756573743A203078257824
:103E000000000000FC6D0020436F6E6E65637465FA
:103E10006400000016BA0F004661696C7572652077
:103E2000746F2075706461746520636F6E6E656376
:103E300074696F6E20706172616D65746572733A3A
:103E40002030782578000000C8BF0F0052656365F8
:103E50006976656420424C455F4741505F45565442
:103E60005F444154415F4C454E4754485F55504470
:103E70004154455F524551554553542E00000000B2
:103E8000526563656976656420424C455F474150E1
:103E90005F4556545F444154415F4C454E4754483A
:103EA0005F555044415445202825752C206D61787C
:103EB0005F72785F74696D65202575292E0000009A
:103EC000526563656976656420424C455F474150A1
:103ED0005F4556545F5345435F504152414D535FD8
:103EE00052455155455354004343434420666F7235
:103EF0002073657276696365206368616E676564C7
:103F0000206973203078253034780000526563656D
:103F10006976656420424C455F4741505F45565481
:103F20005F5048595F555044415445202852583AF3
:103F300025642C2054583A25642C207374617475C0
:103F4000733A2564290000005265636569766564EB
:103F500020424C455F4741505F4556545F50485999
:103F60005F5550444154455F524551554553542E79
:103F700000000000436F756C64206E6F74206861F0
:103F80006E646C65206F6E5F6374726C5F70745FDB
:103F900077726974652E206572725F636F64653A2B
:103FA0002030782530347800526563656976656421
:103FB00020424C455F4741505F4556545F5345434F
:103FC0005F494E464F5F52455155455354000000DE
:103FD00046696E69736865642068616E646C696EB9
:103FE0006720636F6E6E2073656320757064617403
:103FF00065000000007800F00100704738B500202F
:10400000009002F055FE002830D1194C0425194AC1
:10401000208819A105EB004004F02EFB154813DFA2
:10402000002823D120881CA105EB004004F020FBD0
:1040300004F0A8FE002819D1684604F0F9FC002815
:1040400014D120881AA105EB004004F011FB694649
:10405000012004F0F7FC002808D120881AA105EB04
:10406000004004F005FB684604F096FD38BD0000F2
:104070003059002000100F0053657474696E67207A
:10408000757020766563746F72207461626C653A36
:104090002030782530387800456E61626C696E6733
:1040A00020536F66744465766963652E00000000D6
:1040B000436F6E6669677572696E6720424C452072
:1040C000737461636B2E0000456E61626C696E678C
:1040D0002074686520424C4520737461636B2E0028
:1040E00011480421008801EB004010A104F0C0FA3F
:1040F00004F08CFB04F058F90028FBD1114E642524
:104100004FF47A47741C3846A0476D1EFAD1BFF3AE
:104110004F8F0D4801680D4A01F4E06111430160C1
:10412000BFF34F8F00BFFDE76C59002052657365E8
:104130007474696E6720626F6F746C6F616465720E
:104140002E00000090B80F000CED00E00400FA050E
:104150002DE9FC410646C0074FF000050ED0104F78
:1041600000240122385D009500231146019503F0DB
:10417000CBFF641C042CF4D300F064F8B0070DD519
:10418000074E0024361D0022305D032300951146A2
:10419000019503F0B9FF641C042CF4D3BDE8FC8145
:1041A00086B80F0010B50446042803D305A12120CA
:1041B000FFF7A8F90E480121005DBDE8104004F0AA
:1041C00019B800002E2E5C2E2E5C2E2E5C2E2E5C3E
:1041D0002E2E5C636F6D706F6E656E74735C626FB4
:1041E000617264735C626F617264732E63000000BD
:1041F00086B80F0010B50446042803D305A11B2080
:10420000FFF780F90E480021005DBDE8104003F083
:10421000F1BF00002E2E5C2E2E5C2E2E5C2E2E5C0E
:104220002E2E5C636F6D706F6E656E74735C626F63
:10423000617264735C626F617264732E630000006C
:1042400086B80F0010B500242046FFF7ABFF641CB2
:10425000042CF9D310BD00002DE9F8430546861C57
:1042600000208DF8000090460F464FF00109684687
:10427000FFF7B8F81B4C20683860D4E90001401AF9
:10428000A168081A41F21C0167180EE001213846A6
:1042900001F021FA01F0D2F80146384601F01BFA8C
:1042A000D4E90001401AA168081A401C8642EDD8E2
:1042B000B8F1000F03D0052065F3891002E0062055
:1042C00065F39F50A2682168114004EB8101C8602A
:1042D0002068304420609DF80000FFF7CFF8484682
:1042E000BDE8F8839088002010B543689C184460AE
:1042F00021B905E013F8010B01F8010B521EF9D2A8
:10430000012010BD30B482680468531C8360A1543E
:10431000D0E901128A4202D330BC03F0FDBB30BCAD
:1043200070470000034803C8814201D10120704753
:10433000002070479088002010B50548012101F049
:10434000E0F9BFF35F8F08B1002010BD012010BD60
:104350000058002010B5064C2068012803D005A1A4
:104360006D20FFF7CFF8BFF35F8F0020206010BDF6
:10437000005800202E2E5C2E2E5C2E2E5C2E2E5CE5
:104380002E2E5C636F6D706F6E656E74735C6C69FE
:10439000627261726965735C6D757465785C6E726A
:1043A000665F6D74782E6800044900200860044937
:1043B0004FF48060C1F880017047000000A50250F2
:1043C00004E000E003490120086003498002C1F8CD
:1043D0000001704700A5025004E000E070B500F154
:1043E0000806106815460C46202802D248F21450E0
:1043F00070BDFFF7A1FF80B1FFF7E4FF2146304613
:10440000FEF79CF90646FFF7CFFFFFF7A3FF304604
:1044100000F0D4FD060003D004E048F2045070BD63
:10442000202028602021204601F080FF304670BD0A
:1044300010B50830FEF7B2F9BDE8104000F0BEBD7F
:104440002DE9F04700F108090E461446FFF774FF06
:10445000B8B1FFF7B7FF4FF480584546AC4200D8DB
:1044600025462A4631460E48FDF70EF82A460C49E5
:104470004846FEF7ADF90700A4EB05042E4404D02E
:1044800005E048F20450BDE8F087002CE5D1FFF7C5
:104490008BFFFFF75FFF3846BDE8F04700F08EBDA9
:1044A0009C5D002070B50B4800240460BFF35F8F53
:1044B000094D01202860FEF75BFA01002C604FF0E7
:1044C000030004D0052901D148F2035070BD00203B
:1044D00070BD00000058002000A5025001490020D6
:1044E0000860704700A5025010B5040003D10549CB
:1044F000C520FFF707F80448C16B6160006CA0603D
:1045000010BD000060C10F001080002040684968A5
:10451000884201D80120704700207047F0B54FF065
:10452000FF3622B11268D24300230A4D0DE0324615
:10453000FAE7C45C62400824D70700D037462F4012
:1045400087EA5202641EF7D15B1C8B42F1D3D04341
:10455000F0BD00002083B8EDF0B5146906468DB0BB
:1045600020681546271DE0B1022920D00A200090BE
:104570006B4609AA304606F0A3F900280FD009A916
:1045800001A8009A05F0A8FF01AE96E80F0005AE5D
:1045900086E80F00236869683A4605A898470DB079
:1045A000F0BD0DB03046BDE8F04006F009B86946F0
:1045B000304605F09BFF0028F1D0236869683A4631
:1045C000684698470028EAD002980028F5D101985B
:1045D00070600120E3E753685B7813F0C00303D0F9
:1045E000402B03D00020704700F002B8FFF7B4BFA3
:1045F0002DE9FF410B465168064614464878334D75
:1046000000F00F0210F0300055F8225006D01028AC
:1046100006D0202808D0302856D13EE022694DE04F
:1046200061690120087047E0022B28D1042A26D8AE
:104630004FF0010869463046676905F057FF0028CA
:104640001AD009E00B79226913FB00226846A847BB
:1046500070B13878401C3870029820B161683878A1
:104660004A799042EED301987060029860BB02E0F4
:104670004FF00008F7E7404604B0BDE8F081D4E908
:1046800004300F79027817FB023349798A421BD232
:10469000521C02701A46616810E008786169072AA6
:1046A000087009D1606801792069FCF715FF60681E
:1046B0002169806805F035FF2269616804B03046E1
:1046C000AC46BDE8F04160470020D5E7DCBD0F00F7
:1046D00038B51D4901200A68D20301D5000407E05E
:1046E0001A490A6812F0A90F04D0086800F05600B1
:1046F0000860002001F04EFE154C0425D0B11920B1
:104700000090684603F048FDD0F810050099C840B5
:1047100010F0010F13D00D48001F006810F0B10019
:1047200007D020880BA105EB004000BF03F0A0FFDD
:10473000012038BD208810A105EB0040F6E7208855
:1047400016A105EB0040F1E7000400402005004001
:104750006C590020444655206D6F64652072657168
:1047600075657374656420766961204750524547CA
:104770005245542E00000000444655206D6F64657C
:1047800020626563617573652061707020697320B4
:104790006E6F742076616C69642E0000444655206B
:1047A0006D6F6465207265717565737465642076DC
:1047B000696120627574746F6E2E0000FEB5184931
:1047C0000446086808B1401E08601648D4E9015341
:1047D00000880426227806EB00409DB10E6821690E
:1047E0000296CDE900312B46012A16D00EA210A167
:1047F00003F064FF6169002911D0E06803B0BDE8EF
:10480000F040084709680091012A04D006A217A1C8
:1048100003F041FFEEE71FA2F9E71EA2E7E7FEBDA6
:10482000205800203859002065726173650000002F
:10483000466C617368202573206661696C6564202D
:104840002830782578293A20616464723D25702CDF
:10485000206C656E3D307825782062797465732C04
:104860002070656E64696E6720256400466C617314
:104870006820257320737563636573733A206164E0
:1048800064723D25702C2070656E64696E6720250A
:1048900064000000777269746500000010B5082894
:1048A0001BD2DFE800F004121A1A1A041A040120BD
:1048B000FFF74EFC0020FFF79DFC0120FFF79AFC5C
:1048C000BDE810400220FFF76DBC0120FFF76AFC35
:1048D000BDE810400220FFF78DBC10BD10B50446A6
:1048E000032806D0042C04D0062C0ED0072C04D1AB
:1048F0000BE00749074801F0FFF807480168002965
:1049000005D02046BDE810400847FFF7E9FB10BD81
:10491000AD510F00C0D40100B857002010B50446B7
:10492000062802D1002002F0A5FD044801680029F4
:1049300003D02046BDE81040084710BD04580020B1
:1049400010B50021024800F0DCFE80F3100010BD1D
:10495000AC9800204FF4A07202EB810189B200F004
:104960003BBA0068D0F80405704700002DE9F04715
:1049700016460D46040003D136492F20FEF7C2FD2E
:104980001DB934493020FEF7BDFD1EB93149312033
:10499000FEF7B8FD60793049DFF8BC80DFF8BC90E5
:1049A00041F82060617908F1040808EBC100007942
:1049B00038B10824B9F80000022101EB004028A119
:1049C00043E02E882768B6F5805F03D32DA1FD2034
:1049D000FEF798FDC7F80865AD7894F90460A81E45
:1049E000022806D3681F032803D331A14520FEF710
:1049F00089FD002E4FEA451006DA06F00F0101F19D
:104A0000E02181F8140D03E006F1E02686F80004A9
:104A100094F90410012201F01F0302FA03F049097E
:104A2000890001F1E021C1F88002C1F8000161793B
:104A300008EBC1010A71617948F83140B9F800000A
:104A4000032101EB0040002424A103F011FE2046C5
:104A5000BDE8F08710C40F007C580020505900209A
:104A600052544320696E7374616E636520616C7289
:104A70006561647920696E697469616C697A6564DD
:104A80002E0000002E2E5C2E2E5C2E2E5C2E2E5C18
:104A90002E2E5C6D6F64756C65735C6E7266785CEF
:104AA00068616C2F6E72665F7274632E680000001E
:104AB0002E2E5C2E2E5C2E2E5C2E2E5C2E2E5C69F5
:104AC0006E746567726174696F6E5C6E7266785C35
:104AD0006E7266785F676C75652E68005254433A53
:104AE00020696E697469616C697A65642E000000E2
:104AF00090F90400012100F01F029140400980005C
:104B000000F1E020C0F8001270470A46022100F0D0
:104B10004FB94FF4827100F05FB9000010B5040086
:104B200003D104496120FEF7EDFC206801210160FA
:104B300010BD000010C40F0010B5040003D10449DB
:104B40006720FEF7DFFC20680121416010BD0000F6
:104B500010C40F002DE9F843994616460F4605008C
:104B600003D12B498620FEF7CDFC29684FF4803411
:104B70004FF4A070BC4000EB870080B226F07F4667
:104B8000C1F808432968C1F84843296800220A503F
:104B900008580090286800EB8701D1F84005C1F85B
:104BA00040652968D1F804151A4F401A20F07F405B
:104BB0004FF00408012809D1398808EB014016A1FB
:104BC00003F056FD21494FF4046088472868C0F877
:104BD00044432968D1F80435F01A20F07F400202DE
:104BE00001D540F07F40C9F1000290420BDD022860
:104BF00009DC3988324608EB014015A103F043FD7A
:104C00000D20BDE8F883C1F804430020F9E7000057
:104C100010C40F00505900205254433A2044656C90
:104C2000617920696E74726F647563656420647560
:104C30006520746F207269736B206F6620707265D7
:104C40002D666972696E672E0000000071BB0F004F
:104C50005254433A2057696E646F77656420636FDE
:104C60006D70617265207365742074696D656F7510
:104C70007420286162735F76616C75653A25642CD7
:104C800020636F756E7465723A2564292E000000EA
:104C90002DE9FC4180461F4615460E4600240D486E
:104CA00000F016FD38B11120BDE8FC8106EB0430A0
:104CB00003F084FE641CAC42F8D1064800F0FFFC0F
:104CC000CDE90057334600220221404600F02AF881
:104CD0000020E9E7885800202DE9F843104D0F46E1
:104CE00080461E4691466946286800F0BCFC0400D8
:104CF00014D01C21FCF7F0FB01202071C4F81490A3
:104D0000380BC4F80080C4E902606946286800F0E6
:104D1000CBFC05F0B5FD0020BDE8F8830420FBE7DF
:104D2000B4BB0F002DE9F04387B00446DDE90E89DE
:104D300080681D4616460F4600280BD0182168468D
:104D4000FCF7CAFB02A88DF8007080E86003A16838
:104D50006846884707B0BDE8F08330B50446006870
:104D600087B00D46806800281FD018216846FCF7E0
:104D7000B3FB0195A0680590207910B1012810D1EE
:104D800007E001208DF8000020690290E0680390A0
:104D900005E002208DF80000E068000302906069E1
:104DA0000490206881686846884707B030BD0000DD
:104DB00070B516460C46050003D10649B920FEF72A
:104DC000A1FB2868C0F84443002E02D02868C0F830
:104DD000044370BD10C40F0038B50C46050003D164
:104DE0000749CA20FEF78EFB2868015929B1002126
:104DF000015100590090012038BD002038BD00004D
:104E000010C40F000B2803D30B38C0B200F00AB84F
:104E1000704700000249002208780A7070470000BD
:104E200024580020014908700B20704724580020A6
:104E30000149012008707047F95700202DE9FE4311
:104E400007004FF02000904689464FF0010602907F
:104E500004D12A494FF4FA70FEF754FB284C04257C
:104E6000434620884A4605EB004026A103F00BFC90
:104E700002A93348CDE9000143464A463149A0F52D
:104E80009A7001F063F9020007D02088012101EB3C
:104E900000402DA103F0F0FB2CE007F16F01202270
:104EA0000F462748FCF72AFB28B32088022101EB94
:104EB000004032A103F0DCFB208837A105EB004065
:104EC00003F0D6FB2088202205EB0040394603F092
:104ED0007BFB208835A105EB004003F0C9FB20884F
:104EE000202205EB0040164903F06EFB03F05CFA4C
:104EF0000028FBD100263046BDE8FE8338C30F00F2
:104F00004859002048617368207665726966696354
:104F10006174696F6E2E204669726D7761726520CB
:104F2000737461727420616464726573733A2030C3
:104F30007825782C2073697A653A203078257800B6
:104F40001C850020CCB80F00436F756C64206E6F19
:104F5000742072756E206861736820766572696668
:104F600069636174696F6E20286572725F636F6434
:104F7000652030782578292E00000000486173688C
:104F800020766572696669636174696F6E20666117
:104F9000696C65642E000000457870656374656413
:104FA00020465720686173683A00000041637475B9
:104FB000616C20465720686173683A0010B50F4C49
:104FC00048F20351031B48F21652A04211D007DCED
:104FD00000280AD00A4BC01808D0012804D10BE0E1
:104FE0000A2B01D00D2B07D0104610BD48F20150FE
:104FF00010BD48F2025010BD084610BD0202F0007C
:1050000000FE0FFF2DE9FC5F0646DFF804A198467D
:1050100015460F464FF0040BB1420BD1BAF8000011
:1050200033460BEB00403A463AA103F02CFB00203C
:10503000BDE8FC9F04D243494FF02900FEF762FA15
:10504000B8F1000F03D13F492A20FEF75BFA300583
:1050500003D03C492B20FEF755FAB81B040B03D1B3
:1050600038492E20FEF74EFA0020009005F6FF701A
:105070004FEA103900F024FF4046A04500D2044614
:10508000A04641E04946C14504D808462C46CDF823
:10509000049004E040464FEA0834CDF8048001460D
:1050A0000022304601F096FC0028C1D10094BAF8E5
:1050B000001033460BEB01403A4623A103F0EBFA14
:1050C000601E00F00300221A002339463046D21C2D
:1050D00001F030FD0028ABD101992448A9EB01096A
:1050E0002D1B016B2644214401632744002002F05C
:1050F0000BF9009040B1BAF80000012101EB00402B
:105100001BA103F0B5FA01E0002DBBD100988FE799
:105110006C5900204E6F20636F7079206E65656456
:105120006564207372635F616464723A203078252D
:10513000782C206473745F616464723A203078253F
:1051400078000000D4BE0F00436F7079696E67204D
:105150003078257820746F20307825782C2073697A
:105160007A653A2030782578000000001080002011
:105170004661696C656420746F207772697465207C
:10518000696D61676520636F7079696E6720707201
:105190006F677265737320746F2073657474696EC2
:1051A000677320706167652E0000000004480321CA
:1051B000008801EB004003A103F05AFAFEF790FFCC
:1051C0006C590020496E6163746976697479207442
:1051D000696D656F75742E0001494160002070474C
:1051E00088BB0F0010B50B4941600B4800F070FA06
:1051F00068B903F019FE08491C234FF4EE720874D5
:105200000448A1F5EE71001F006800F019FA0020B3
:1052100010BD0000B8BB0F007C8700202DE9FC5FAB
:105220000E008346DDE90C47C6F100009846924621
:10523000814600D40846012503E000BF90FBFAF048
:105240006D1C5045FADAA84500D9454624B1002E18
:1052500001DB780700D5641EB80702D5B8F1000F4E
:105260000AD0F80708D13CB1A54205D22021584602
:10527000641EFFF747F8F6E7002E02DA4E462D21AE
:1052800002E0780703D52B215846FFF73BF807F0DB
:10529000030002280BD1B8F1000F08D13CB1A542A0
:1052A00005D230215846641EFFF72CF8F6E7CDE909
:1052B0000047434652463146584606F023F9BDE8BA
:1052C000FC9F000010B5024600201268930702D030
:1052D000530702D410BD500719D502F0030001286E
:1052E00007D002280BD00D494FF49170FEF70AF950
:1052F0000BE0C2F383100B68801C184404E0022307
:10530000086803EB925210440860012010BD086841
:1053100000EB9253C2F38910401CEEE730C90F0036
:1053200002480068002800D00120704788580020FB
:105330000248007A002800D0012070477C870020B6
:1053400038B54FF440531A4A5D6800F50051954254
:1053500004D04868904201D1012400E00024954225
:1053600024D14868904221D11878142801D95A696B
:1053700000E000220F48B2FBF0F30A78142A01D9AA
:10538000496900E00021B1FBF0F0834203D0012421
:1053900009A2009002E0002409A200900A4803211B
:1053A000008801EB004009A103F075F9204638BDE3
:1053B000DBE5B15140420F006D616A6F7200000081
:1053C0006D696E6F7200000048590020536F66745B
:1053D00044657669636520757064617465206973DE
:1053E00020612025732076657273696F6E20757059
:1053F000646174652E2043757272656E743A20255F
:10540000642E204E65773A2025642E0070B505463F
:1054100008680C464A6886682846314604F0A2FFB0
:105420006068286104F10C00686170780221B1EBBA
:10543000901F01D1241D2C6170BD00002DE9FF419A
:105440000026264800F041F92448001F074600F0D6
:105450003CF9234C60680090A56800E0009869461C
:10546000284004EB80000C30FFF72CFF0028F5D11A
:1054700001AA009901EA050304EB8303491CDB68D8
:1054800042F82030401C00910228F2D3019800F02D
:10549000030001281AD002280ED012494FF4AF7031
:1054A000FEF730F8384600F00DF908B1009860605A
:1054B00004B03046BDE8F0810198032101EB905023
:1054C0000099BDF80A6001EB900005E00198BDF875
:1054D0000A60C0F3831008440090E3E7A898002016
:1054E0009088002030C90F0070B500224FF4805121
:1054F000104600F009FBC8B912480022C0F57E2111
:1055000000F002FB90B94FF400410F4803F03AF964
:1055100002F034FF0D4C03250DA1208805EB00405F
:1055200003F0A6F80D4800F00BFC08B1FDF738FEBB
:1055300000F0FAF920880AA105EB004003F098F882
:10554000002070BD00100F00E5320F006C590020E4
:10555000496E73696465206D61696E009D480F0036
:105560004166746572206D61696E00002DE9F05F1F
:10557000C7888A46191D1646B1FBF7F2B1FBF7F54D
:1055800007FB121999193944C91CB1FBF7F10446FC
:105590004079C9B2DDF828B0884206D21749942074
:1055A000FDF7B0FF01E024686D1E002DFBD1A84679
:1055B000A7EB0905B5421AD81CE000BFBBF1000FEC
:1055C00006D004EB09010AEB08002A46091D05E094
:1055D00004EB09000AEB08012A46001DFBF754FF03
:1055E0002468761B4FF00009A844B74201D935461C
:1055F00000E03D46002EE1D1BDE8F09F54C40F000D
:1056000030B5024659B103F0E9F80021074C09E032
:1056100004EB810315685B88AB4202D11160002066
:1056200030BD491C8142F3D3052030BD24590020F0
:1056300010B5FBF73EFE08B1002010BD112010BDD3
:1056400010B531B1B2FBF3F403FB14241CB10920F3
:1056500010BD0E2010BD016000214160816082817B
:10566000C381084610BD70B50C460546FBF7D6FD54
:10567000002802D021882868084470BD10B50A8827
:1056800049888A4203D1FBF70BFE012010BD0020A0
:1056900010BD70B50C460546FBF7E5FD002802D0AD
:1056A00061882868084470BD10B50A8849888A4214
:1056B00003D1FBF7CFFD012010BD002010BD00215C
:1056C00000F00FB8002100F012B8012100F01EB860
:1056D000012100F011B808B56A46FBF736FE0098C4
:1056E00008BD08B56A46FBF716FE009808BD08B568
:1056F0006A46FBF710FE08BD08B56A46FBF7FEFDDB
:1057000008BD08B56A46FBF7EDFD08BD08B56A4659
:10571000FBF7F4FD009808BD08B56A46FBF722FECA
:10572000009808BD38B5040003D115A1FE20FDF78F
:10573000E9FE00258DF800506846FDF753FE20680D
:1057400062680168914214D9491E01600D781CB944
:1057500019A1C220FDF7D6FEA08AE16805FB00155D
:105760002068217A0278891A0279C9B28A4200D265
:1057700001719DF80000FDF781FE284638BD00004C
:105780002E2E5C2E2E5C2E2E5C2E2E5C2E2E5C631E
:105790006F6D706F6E656E74735C6C69627261724E
:1057A0006965735C62616C6C6F635C6E72665F628C
:1057B000616C6C6F632E63002E2E5C2E2E5C2E2E81
:1057C0005C2E2E5C2E2E5C636F6D706F6E656E743A
:1057D000735C6C69627261726965735C62616C6C46
:1057E0006F635C6E72665F62616C6C6F632E6300E8
:1057F00038B50C46050004D112A140F22110FDF786
:1058000081FE24B90FA14FF49170FDF77BFE0020BB
:105810008DF800006846FDF7E5FD1DB91749CF205A
:10582000FDF770FEE8682A68211AA88AB1FBF0F13A
:105830001068431C136001709DF80000FDF71EFE08
:1058400038BD00002E2E5C2E2E5C2E2E5C2E2E5C83
:105850002E2E5C636F6D706F6E656E74735C6C6919
:10586000627261726965735C62616C6C6F635C6EBD
:1058700072665F62616C6C6F632E6300B8570F00D5
:1058800010B5040002D0206830B901E00E2010BD30
:1058900017A1D920FDF736FE606818B914A1DA20E7
:1058A000FDF730FEA06818B911A1DB20FDF72AFE34
:1058B000E06818B90EA1DC20FDF724FEA08A18B913
:1058C0000BA1DD20FDF71EFE207A61682268401AD8
:1058D000C0B2116004E0226811684B1C13600870AC
:1058E000401EC0B2F7D221680020087110BD000030
:1058F0002E2E5C2E2E5C2E2E5C2E2E5C2E2E5C63AD
:105900006F6D706F6E656E74735C6C6962726172DC
:105910006965735C62616C6C6F635C6E72665F621A
:10592000616C6C6F632E63002DE9F041184D4FF4EC
:10593000805204272888164607EB004015A102F084
:105940009BFE4FF0E024D4F8802128881FA107EBAC
:10595000004004F5C07402F08FFE60172060C4F8A8
:1059600000016060C4F8040101F0AEF930B128888C
:10597000012101EB004020A102F07AFE02F014FDAB
:105980000028FBD13046BDE8F04100F051B80000DE
:105990006C59002052756E6E696E67206E72665F7C
:1059A000626F6F746C6F616465725F6170705F735A
:1059B00074617274207769746820616464726573BD
:1059C000733A2030782530387800000044697361DC
:1059D000626C696E6720696E74657272757074733B
:1059E0002E204E5649432D3E494345525B305D3A89
:1059F00020307825780000004661696C656420726B
:105A0000756E6E696E67206E72665F6466755F6D37
:105A100062725F6972715F666F72776172645F61F3
:105A20006464726573735F736574282900000000F5
:105A300070B506461F4888B0C0F57F21002200F0EF
:105A400063F8021E4FF0FF3507D01B480121008884
:105A500001EB004019A102F00FFEEFF30580D6E93B
:105A60000046C005C00D4FF0000181F3148881F39A
:105A7000108881F3118881F3138813D020221D49E7
:105A80006846FBF701FD203C202269462046069629
:105A9000FBF7FAFC6FF0060229462046FBF7BAFB3B
:105AA00008B070BD08B0324629462046BDE87040B7
:105AB000FBF7B0BB00100F006C590020436F756CF2
:105AC00064206E6F742070726F7465637420626FEF
:105AD0006F746C6F6164657220616E6420736574AD
:105AE00074696E67732070616765732C2030782548
:105AF000782E000098B80F000A4601460148006859
:105B000005F0B2BCB8B80F0070B50B0502D1B0F506
:105B10007F2F01D9072070BD0AB1062500E00225BC
:105B2000104A114B1468082C01D3042070BD03EBFC
:105B30000416C6F80008C6F80418C6F80858641C0D
:105B4000146003EB0414D4F8F0678642EAD1D4F869
:105B5000F4678E42E6D1D4F8F847AC42E2D1002097
:105B600070BD0000BC57002000E001402DE9F04767
:105B70003D4C04253B4E2088002705EB00403BA10F
:105B800002F076FDB06801280FD0A52816D0AA280B
:105B90001DD0AC28208824D0032101EB00403CA17B
:105BA00002F066FD0020BDE8F08720883FA105EBEC
:105BB000004002F05DFDFDF749FA10E020883EA1AB
:105BC00005EB004002F054FD04F062FF10E0208875
:105BD0003CA105EB004002F04BFDFDF79FFC0246A7
:105BE00008E005EB00403AA102F042FD05F020F884
:105BF000024601274FF0010932B12188B36809EB51
:105C0000014037A102F03FFD304600F055FCDFF8BF
:105C10000481002188F800103F4801F075FB06461A
:105C200098F8000020B93D4940F27910FDF76AFC70
:105C300046B1218809EB014039A102F019FD032684
:105C40003046B0E70126002FFAD0012000F0A2FB79
:105C50000028F5D02088394905EB004002F008FD06
:105C60000226EDE7348000206C590020456E7465F3
:105C700072206E72665F626F6F746C6F61646572C2
:105C80005F66775F61637469766174650000000028
:105C90004E6F206669726D7761726520746F206146
:105CA000637469766174652E0000000056616C694A
:105CB000642041707000000056616C696420534498
:105CC0000000000056616C696420424C0000000036
:105CD00056616C6964205344202B20424C00000024
:105CE00041637469766174696F6E206661696C6581
:105CF000642077697468206572726F722025642051
:105D00002862616E6B20636F64653A203078257875
:105D100029000000F9570020314E0F00D4BE0F00BB
:105D2000436F756C64206E6F7420777269746520A0
:105D300073657474696E67732E0000006CBF0F008A
:105D4000F8B5354C05460426208834A106EB004002
:105D500002F08EFC3748056019200090684602F07A
:105D60001BFA009A344900EB8200C0F800170020AB
:105D700001F0FCF9002842D1FFF7F8FE20B101281C
:105D800020D002283BD104E02C4DFEF7A1FC10B935
:105D900032E042F2107500F093F8294A20211820D1
:105DA000FDF78AFA08B1FDF7FBF92648016811F002
:105DB000B10F03D0016801F04E01016000F050FF07
:105DC000E8B901E0FEF78CF91F492846FFF794FE79
:105DD0001E4800F0FDFE90B920881DA106EB004092
:105DE00002F046FC00F05AF8FDF746FA02F0DCFA41
:105DF0000028F7D141DFF5E701F078F908B1032079
:105E0000F8BDFFF791FD2088012101EB004014A1AE
:105E100002F02EFCF3E700006C590020496E206E62
:105E200072665F626F6F746C6F616465725F696EDA
:105E300069740000B85700200C000300C0D40100B2
:105E40007C5900201C050040AD510F00DD480F00BB
:105E5000456E746572206D61696E206C6F6F7000A5
:105E600053686F756C64206E6576657220636F6D24
:105E70006520686572653A204166746572206E72AD
:105E8000665F626F6F746C6F616465725F61707082
:105E90005F737461727428290000000010B503F06C
:105EA000CBF9002803D0BDE8104005F03DBC10BD83
:105EB0000A4601460148406805F0D6BAB8B80F0056
:105EC0002DE9F041224C207800283FD103F0B4F9AD
:105ED000204E03274FF0010800282FD01E480068ED
:105EE0001EA1450930882A4607EB004002F0C4FB9A
:105EF00005EB4500850842F21070854201D2012071
:105F000000E00020607005F00FFC607820B91248B6
:105F100008300068C0070AD030882A4607EB0040E6
:105F200014A102F0A9FB1F492846FFF7C1FF4FF05B
:105F3000E0214FF48030C1F8000105E030881AA15B
:105F400007EB004002F094FB84F80080BDE8F0818C
:105F5000FA5700202C5900200405014057445420D2
:105F6000656E61626C6564204352563A2564206D0B
:105F7000730000005374617274696E67206120744D
:105F8000696D657220282564206D732920666F7203
:105F90002066656564696E67207761746368646F05
:105FA000672E000065B70F00574454206973206EB8
:105FB0006F7420656E61626C6564000070B50446A4
:105FC0000D462022083000F077F9202205F120014B
:105FD00004F1280000F070F9002070BDF0B599B010
:105FE0000D4621491E9E944607460160202B00D392
:105FF00020231C461A46614611A800F05DF92022B4
:10600000314601A800F026F918480121FFF779FB75
:10601000BFF35F8F002618B148F2045019B0F0BDED
:10602000FEF7D0F911AB01AA05F10801384600943A
:10603000FCF770FB0446FEF7B7F90C4D2868012801
:1060400003D00BA16D20FDF75DFABFF35F8F2E60CB
:1060500044B11448C44202D148F24250DEE748F24B
:106060001650DBE70020D9E7DD55AABB0058002019
:106070002E2E5C2E2E5C2E2E5C2E2E5C2E2E5C6325
:106080006F6D706F6E656E74735C6C696272617255
:106090006965735C6D757465785C6E72665F6D744E
:1060A000782E68007CF70FFF70B516460C46054643
:1060B00000F0E9F800280ED1AA791946304600F020
:1060C000EFF8002807D131462046FFF777FF002878
:1060D00001D10149216070BD7052464D2DE9F84F44
:1060E0006C460E46D4E90A7905469A46904616490A
:1060F000304600F0BCF80028A54611D1706849462A
:1061000040794200384600F0CBF80028A54607D178
:10611000B8F1000001D02DB107E0A54648F21050BB
:10612000BDE8F88FAAB06D464DB182B00246534625
:10613000314628460097FFF751FFA546F0E748F2A1
:106140001550A546ECE700007052464D2DE9F04190
:106150001D46DDE906871646044600F02DF80028A6
:106160000DD12A463146204600F03CF8002806D1E1
:106170003A4641462046BDE8F04100F002B8BDE88D
:10618000F08170B515460E46044605F0BDFA0028AC
:1061900007D13EB160682968C268914205D248F2D1
:1061A000145070BD48F2135070BD83682A463146C2
:1061B0002046BDE87040184710B550B161B141604C
:1061C000096804468847002802D10548206000205D
:1061D00010BD48F2015010BD48F2105010BD000033
:1061E0006E52464870B515460E46044605F08CFAC8
:1061F00000280BD146B155B160682A463146436844
:106200002046BDE87040184748F2105070BD00208D
:1062100070BD00002DE9F0410B480C4D0C4F401BA8
:10622000C60801203870002406E000BF55F834008D
:106230008047002805D1641CB442F7D3022038708F
:106240000020BDE8F0810000B0CE0F00A8CE0F0006
:10625000FC57002070B514460D46064600F02CF899
:10626000291930192246BDE8704000F025B828B140
:106270000068884205D048F24050704748F21050FC
:1062800070470020704728B139B10022C1E90020D1
:106290001046704748F21050704748F2135070474C
:1062A00020B1914205D048F21150704748F2105089
:1062B000704700207047000070B516460C46050078
:1062C00003D10AA11F20FDF71DF91CB907A1202049
:1062D000FDF718F9A919491E04E000BF14F8010BD5
:1062E00001F80109A942F9D270BD00002E2E5C2EE2
:1062F0002E5C2E2E5C2E2E5C2E2E5C636F6D706FCE
:106300006E656E74735C6C69627261726965735CF0
:1063100063727970746F5C6E72665F6372797074A9
:106320006F5F7368617265642E63000070B50D461F
:10633000040003D107A10D20FDF7E4F86019401E09
:1063400005E02178027804F8012B00F80119A04239
:10635000F7D270BD2E2E5C2E2E5C2E2E5C2E2E5C67
:106360002E2E5C636F6D706F6E656E74735C6C69FE
:10637000627261726965735C63727970746F5C6E6E
:1063800072665F63727970746F5F7368617265645F
:106390002E6300002DE9F041174C074604252088A4
:1063A00016A105EB004002F063F91B4E306A01288C
:1063B00004D0208819A105EB00400FE09FB1F069DF
:1063C00088B100F055F80022B169FEF7A7F8F1692D
:1063D000814208D0208819A105EB004002F048F95D
:1063E0000020BDE8F081208819A105EB004002F0F3
:1063F0003FF90120F5E700006C590020456E7465F7
:1064000072206E72665F6466755F6170705F69733B
:106410005F76616C696400001080002052657475BD
:10642000726E2066616C736520696E2076616C699E
:10643000642061707020636865636B0052657475D9
:10644000726E2066616C736520696E204352430052
:1064500052657475726E20747275652E204170706D
:10646000207761732076616C69640000AFF300806F
:106470004FF44050074A4168914207D18068411E5D
:10648000C1F30B01401A00F6FF7070474FF48050C3
:1064900070470000DBE5B15100B5FFF7E9FF0549A2
:1064A00089690A18401E0844C0F30B00101A00F650
:1064B000FF7000BD108000200021016041608160FC
:1064C0000148016370470000108000202DE9FF5F44
:1064D0007E4C04257EA1208805EB004002F0C8F820
:1064E000208883A105EB0040009A02F0C5F80198CE
:1064F00008B185A200E086A2208887A105EB0040B4
:1065000002F0BAF8029808B17FA200E080A22088C9
:1065100086A105EB004002F0AFF8039808B17AA21B
:1065200000E07BA2208885A105EB004002F0A4F8E2
:106530004FF4405041688748814201D172A200E087
:1065400073A2208884A105EB004002F095F8208812
:1065500085A105EB004002F08BF8874E208887A1CB
:1065600005EB0040B369326A02F08DF820888BA1F8
:1065700005EB0040736AF26A02F085F84FF00008FC
:10658000DFF838B2A146AA461AE00127C0B10128B7
:1065900020D0B8F1020F2CD08949A420FCF7B2FF1B
:1065A00000255D4503D98649A920FCF7ABFF854846
:1065B0000099401BA0F5405088421DD201261CE0E6
:1065C000FFF76AFF0546029888B16B48006A012808
:1065D0000BD00CE0FFF74CFF0546039828B94FF4A9
:1065E000405041685B48814201D00127D9E700272C
:1065F000D7E74FF48055D4E700260198B9F800108A
:1066000046EA00040AEB014042466FA102F034F86A
:10661000B9F800102A460AEB01406EA102F02CF8EE
:106620000EB139A200E03AA2B9F800104D460AEBCB
:1066300001406EA102F020F80FB133A200E034A2B5
:106640002888A94655460AEB00406EA102F014F8CE
:106650000CB12DA200E02EA2B9F800006EA105EB4E
:10666000004002F009F8BC4308D0B8F1020F05D28F
:1066700008F10100C0B28046022886D95EB1B9F89F
:106680000000022101EB004068A101F0F1FF0420AD
:1066900004B0BDE8F09FB8F1000F0AD0B9F80010BF
:1066A0000AEB01406CA101F0E3FF33481830FFF71B
:1066B00003FF314A002010610120506102F12400E3
:1066C000FFF7FAFE009850620020E1E76C590020C5
:1066D000456E746572206E72665F6466755F636195
:1066E0006368655F707265706172652829000000DB
:1066F00072657175697265645F73697A653A203095
:106700007825782E00000000747275650000000086
:1067100066616C736500000073696E676C655F622B
:10672000616E6B3A2025732E000000006B6565706A
:106730005F6170703A2025732E0000006B656570F4
:106740005F736F66746465766963653A2025732E9E
:1067500000000000DBE5B15153445F505245534502
:106760004E543A2025732E0042616E6B20636F6E8B
:1067700074656E74733A00001080002042616E6B85
:10678000203020636F64653A203078253032783AC3
:106790002053697A653A20307825780042616E6B23
:1067A000203120636F64653A203078253032783AA2
:1067B0002053697A653A20307825780000E00E0091
:1067C000ACC10F0000100F00706173733A20256494
:1067D0002E00000063616368655F616464726573C5
:1067E000733A20307825782E0000000063616368DA
:1067F000655F746F6F5F736D616C6C3A2025732EEB
:10680000000000006B6565705F6669726D7761728C
:10681000653A2025732E000064656C6574655F6DB4
:106820006F72653A2025732E0000000041626F727E
:1068300074696E672E2043616E6E6F742066697492
:10684000206E6577206669726D77617265206F6E64
:106850002064657669636500496E76616C69646180
:1068600074696E67206170702E00000070B50C4670
:10687000050004D1224940F22D10FCF743FE24B953
:106880001F494FF49770FCF73DFE2A7804201D49FC
:10689000092A2DD2DFE802F02C052C0B182C1E2C17
:1068A000120021462846BDE8704002F0CDBC0988A0
:1068B00000EB014014A101F0DBFE14E02146284664
:1068C000BDE8704002F05ABD21462846BDE8704040
:1068D00002F0F6BC098800EB014014A101F0C8FEEB
:1068E0004FF48070E0602046BDE87040FDF7FCBDCD
:1068F000BDE87040024940F24D10FCF703BE0000B5
:1069000060C10F003C59002048616E646C65204EE8
:1069100052465F4446555F4F505F4352435F474581
:10692000542028636F6D6D616E64290048616E6448
:106930006C65204E52465F4446555F4F505F4F4254
:106940004A4543545F53454C4543542028636F6D7B
:106950006D616E642900000070B50E46040004D11C
:106960001B4940F24620FCF7CDFD26B9184940F2FC
:106970004720FCF7C7FD20780125092820D2DFE851
:1069800000F01F051F0F141F1A1F0A003146204672
:1069900002F0C6FD19E03146204603F00BF814E082
:1069A0003146204602F080FD0FE03146204602F0DD
:1069B000CBFE054609E03146204602F0B3FF04E075
:1069C00003494FF41A70FCF79DFD284670BD000086
:1069D00060C10F002DE9F843134C0746134E2068A1
:1069E0000D46009030880421904601EB00402B4674
:1069F0003A460FA101F04FFE43462A4639461C484D
:106A000001F0DEF905000AD03088022101EB0040D8
:106A10002A4618A101F030FE2846BDE8F883206818
:106A2000401C2060F8E70000205800203859002062
:106A30006E72665F6673746F726167655F657261BF
:106A4000736528616464723D307825702C206C6514
:106A50006E3D2564207061676573292C2071756512
:106A600075652075736167653A2025640000000034
:106A7000105900206E72665F6673746F726167658D
:106A80005F65726173652829206661696C656420A1
:106A900077697468206572726F7220307825782E5D
:106AA000000000000B4910B504220988002802EB01
:106AB0000142104604D008A101F0DAFD104903E0BC
:106AC00010A101F0D5FD1949BDE810400022184879
:106AD00001F0D6B938590020496E697469616C6952
:106AE0007A696E67206E72665F6673746F72616733
:106AF000655F7364206261636B656E642E000000E5
:106B0000C4BB0F00496E697469616C697A696E670C
:106B1000206E72665F6673746F726167655F6E7612
:106B20006D63206261636B656E642E0094BB0F0021
:106B3000105900202DE9FC47154C8046154E206861
:106B40000F46CDE90020308804219946154601EB17
:106B500000403B464246104901F0A6FD2B463A460E
:106B600041460E48CDF8009001F052FA05000AD0D7
:106B70003088022101EB00402A4609A101F07CFD8A
:106B80002846BDE8FC872068401C2060F8E700002C
:106B90002058002038590020A8C00F0010590020AC
:106BA0006E72665F6673746F726167655F77726934
:106BB00074652829206661696C656420776974684A
:106BC000206572726F7220307825782E00000000E8
:106BD00070B51049104D08602888032101EB004072
:106BE0000EA101F045FD0020FDF798FE104800F0D1
:106BF0009FFC040009D02888012101EB00402246B7
:106C00000CA101F039FD204670BDBDE87040084878
:106C100000F0C8B8045800206C590020456E746517
:106C200072696E6720444655206D6F64652E0000C2
:106C30001D490F00436F756C64206E6F7420696E80
:106C40006974616C697A6520444655207472616E7E
:106C500073706F72743A20307825303878000000F5
:106C6000054810B50088042101EB004003A101F0A4
:106C7000FFFC002010BD00006C590020696E2077D9
:106C800065616B206E72665F6466755F696E6974BC
:106C90005F757365720000001FB58908002201ABA3
:106CA000009283E80700684618DF04B010BD0000BA
:106CB0001FB5044B0FCB8DE80F00684618DF04B0FA
:106CC00010BD000018BB0F0070B50A4C04254FF42E
:106CD0008056208808A105EB004001F0C9FCE806B9
:106CE0000BA106602088002605EB004001F0C0FCE7
:106CF000304670BD6C59002072756E6E696E6720EB
:106D0000697271207461626C6520736574000000A3
:106D100041667465722072756E6E696E6720697265
:106D200071207461626C65207365740070B50E46E5
:106D30000178124C062901D0012901D1017C217072
:106D40002178012501290FD0022911D00C480121F9
:106D5000008801EB00400BA101F08AFC00202070AC
:106D600005207070284670BD3146FFF77FFDF9E7BA
:106D70003146FFF7F1FD0546F4E7000028580020F2
:106D80003C590020496E76616C6964206F626A65C7
:106D90006374207479706520696E20726571756501
:106DA00073742E0010B5040011D00120FFF77AFE95
:106DB00000280BD100F016FC00F02CFD48B1094969
:106DC000081F00F09DFC012803D0032010BD072000
:106DD00010BD04480838C4600020FEF723F80020E6
:106DE00010BD00003058002010B5816879B1094A03
:106DF0001821FCF7F1F9040007D0074802210088A8
:106E000001EB004005A101F033FC204610BD072036
:106E100010BD0000396E0F003C59002053636865B7
:106E200064756C65722072616E206F7574206F6678
:106E30002073706163652100AFF30080F0B50446F4
:106E4000806887B020B946494FF42870FCF75AFB98
:106E5000182244496846FAF717FB20788DF800009D
:106E600022780426404F414D0D2A5AD2DFE802F025
:106E7000075237525259523E522D0F284800288847
:106E80003BA106EB004001F0F3FB012024E0288841
:106E900040A106EB004001F0EBFB4FF08050D0F832
:106EA00000110191D0F804110291D0F80C1189025F
:106EB0000491D0F8101189020391006905903AE01D
:106EC0006946204602F064FE35E028883AA106EBC8
:106ED000004001F0CDFB207C8DF804002BE02888D9
:106EE0003BA106EB004001F0C3FB24E0288841A150
:106EF00006EB004001F0BCFB208AADF804001AE06C
:106F0000288843A106EB004001F0B2FBF968072096
:106F1000884710E069462046FFF708FF58B907B0D8
:106F2000F0BD2888032101EB00403FA101F0A4FB44
:106F300002208DF8010028889DF8012006EB004012
:106F400041A101F099FBD4E90112684690479DF8F0
:106F500001000128E3D0F96805208847DFE7000039
:106F600060C10F0040BB0F00285800203C59002092
:106F700048616E646C65204E52465F4446555F4FD3
:106F8000505F50524F544F434F4C5F5645525349F8
:106F90004F4E000048616E646C65204E52465F445F
:106FA00046555F4F505F48415244574152455F56E6
:106FB000455253494F4E000048616E646C65204E47
:106FC00052465F4446555F4F505F50494E47000060
:106FD00048616E646C65204E52465F4446555F4F73
:106FE000505F524543454950545F4E4F5449465FA8
:106FF0005345540048616E646C65204E52465F44B0
:1070000046555F4F505F4D54555F47455400000053
:1070100048616E646C65204E52465F4446555F4F32
:10702000505F41424F525400496E76616C69642052
:107030006F70636F64652072656365697665643A35
:1070400020307825782E00005265717565737420A4
:1070500068616E646C696E6720636F6D706C6574D7
:10706000652E20526573756C743A2030782578004F
:1070700038B10549016005494160012101720020D4
:1070800070470E207047000091700F00C9700F000C
:1070900010B50C0001464FF0110007D02278052AE8
:1070A00005D2DFE802F00F050D0F0F000E2010BD16
:1070B000084600F00DF90028F9D10221217010BD19
:1070C000112010BD082010BD0246082041B10B78E8
:1070D000022B04D1022A05D0032A00D111207047C7
:1070E0000E207047002003220A70704770B50F48C9
:1070F0000024D0F85C11491C03D1D0F89C01401C3D
:1071000011D00B480421008801EB004009A101F0D7
:10711000AFFA4FF47F25284601F050FC572203496F
:10712000284601F063FC204670BD0000108000205E
:107130004459002045726173696E672073657474E9
:10714000696E677320706167652061646469746942
:107150006F6E616C20646174612E00000022582102
:107160000148FDF7DBB90000148000202DE9F04153
:107170001F4C0546042620881EA106EB004001F0A6
:1071800077FA2846FFF78EFC02004FF0010504D085
:10719000208821A105EB004023E04FF4DC78424633
:1071A00028492948FAF770F9274F3868401C04D05D
:1071B000FFF7D4FF3968814218D0208823A106EB5D
:1071C000004001F055FA41461F48FAF785F90020C2
:1071D0007D6000F099F8020008D0208823A105EB1B
:1071E000004001F049FA0320BDE8F0810020FBE7F0
:1071F0004059002043616C6C696E67206E72665F57
:107200006466755F73657474696E67735F696E69D0
:107210007428292E2E2E00006E72665F6466755FDC
:10722000666C6173685F696E69742829206661699C
:107230006C65642077697468206572726F723A2099
:107240002578000000F00F00108000205265736563
:107250007474696E6720626F6F746C6F61646572BD
:107260002073657474696E67732E00006E72665FBA
:107270006466755F666C6173685F777269746528B0
:1072800029206661696C656420776974682065727D
:10729000726F723A2025780010B528B14022034958
:1072A000FAF7F2F8002010BD0E2010BD5CF10F00BF
:1072B00010B5064C00223C21201DFDF72FF9216856
:1072C000814201D1012010BD002010BD5CF10F00F2
:1072D00070B50C4D0400D5F85C0105F5AE7503D012
:1072E000401C03D0082070BD0E2070BD00223C2140
:1072F000201DFDF713F9206010222146284629DFC2
:1073000070BD000000F00F002DE9F04105464FF47C
:10731000DC773A4621492248FAF7F0F8214C042656
:107320000028208806EB004015D01FA101F0A0F92D
:1073300020881A4A06EB004020A101F09DF90022A6
:1073400001211648FFF746FB012668B1208823A1DA
:1073500006EB00401DE02AA101F08AF90DB10020E2
:10736000A8470020BDE8F081FFF7F8FE0C493A4637
:107370000860A1F5DC70FAF787F82B463A463049E9
:107380000648FFF7D7FB0028ECD020882DA106EB9C
:10739000004001F06DF90320E4E7000000F00F0069
:1073A000108000204059002057726974696E672070
:1073B00073657474696E67732E2E2E004572617347
:1073C000696E67206F6C642073657474696E67738F
:1073D0002061743A2030782530387800436F756C1E
:1073E00064206E6F74206572617365207468652017
:1073F00073657474696E677320706167652100003E
:107400004E65772073657474696E67732061726569
:10741000206964656E746963616C20746F206F6CA1
:10742000642C207772697465206E6F74206E6565B8
:107430006465642E20536B697070696E672E00005E
:10744000587E0020436F756C64206E6F74207772D5
:1074500069746520746865204446552073657474AA
:10746000696E677320706167652100004FF480507A
:10747000704700002DE9F04782461548154FDFF8A8
:107480005880C01BC608B8F800104FF0040909EB7B
:1074900001400025324611A101F0EEF8002411E070
:1074A00007EBC400416850468847050009D0B8F88A
:1074B00000102B4609EB0140224612A101F0E3F82F
:1074C00002E0641CB442EBD32846BDE8F08700001C
:1074D000B8CE0F00B0CE0F006C5900205368757401
:1074E00074696E6720646F776E207472616E73705A
:1074F0006F7274732028666F756E643A2025642954
:10750000000000004661696C656420746F20736838
:107510007574646F776E207472616E73706F7274BD
:107520002025642C206572726F7220256400000093
:107530002DE9F04782461448144FDFF85480C01BF1
:10754000C608B8F800104FF0040909EB0140002507
:10755000324610A101F090F8002410E057F83410E2
:1075600050468847050009D0B8F800102B4609EBB3
:107570000140224610A101F086F802E0641CB442EA
:10758000ECD32846BDE8F087B8CE0F00B0CE0F0090
:107590006C590020496E697469616C697A696E671B
:1075A000207472616E73706F7274732028666F75C9
:1075B0006E643A20256429004661696C6564207414
:1075C0006F20696E697469616C697A652074726193
:1075D0006E73706F72742025642C206572726F72E6
:1075E0002025640070B5114D114CA86B30B103F02B
:1075F00017FE18B1686A08B1012000E00020207071
:10760000FEF708FE18B10B498E20FBF77BFF4023E5
:10761000094A0A490A48FEF747FD002805D0BDE897
:10762000704004499620FBF76DBF70BD10800020AC
:107630003858002038C30F003CB80F007484002075
:10764000C0B80F002DE9F041134C07460D46E06B22
:10765000A26B01264119914209D9104801210088E5
:1076600001EB00400EA101F003F8032610E00A49E7
:107670002A465C3108443946F9F706FFE06B064AB2
:107680002844E063403229463846FCF747FF20642F
:107690003046BDE8F08100001080002048590020ED
:1076A000496E697420636F6D6D616E64206C6172E8
:1076B000676572207468616E2065787065637465B3
:1076C000642E000070B505004FF0010404D0B5F53C
:1076D000807F03D904240CE003240AE0064900203B
:1076E000064E08702021306306F13800F9F7F4FEE9
:1076F000B563204670BD000038580020108000207F
:107700002DE9F047304C0E468046D4E90E010125A4
:10771000DFF8B8902F46814208D0B9F800002CA1BC
:1077200007EB004000F0A4FF082549E0DFF8BCA00B
:107730009AF8000030B1FEF7AFFEC8F80000606AAA
:1077400030603DE003F06CFD88B3294890F89C1050
:1077500009B9017859B3041D0021C8F8001031603F
:1077600090F89C300A462BB1214C90F83811A03487
:1077700004F1990294F8590003F094FB054601289E
:107780001ED1201D00F0B8F80546012818D18AF84E
:1077900000703146201D03F051FF054601280FD12E
:1077A0004246201D316803F007FF054608E0FFE769
:1077B000B9F800000FA107EB004000F059FF0525C4
:1077C0002846BDE8F08700001080002048590020BE
:1077D000457865637574652077697468206661759E
:1077E0006C7479206F6666736574000038580020E9
:1077F000C88100204661696C656420746F206465EF
:10780000636F646520696E6974207061636B657471
:107810000000000001480078704700003858002040
:107820002DE9F04780462748264D894690F89C0070
:10783000012608B1A43500E008350A46414628462D
:10784000FDF7FCFA204C002760B195F8550058B1BF
:1078500000F00101C0F340024346284602F0FCFE5E
:10786000C8B114E0172617E00120E0621748042190
:10787000008801EB004016A100F0FAFE276295F89F
:107880008F0010B195F8900008B96868A060A06CEE
:10789000C4E9099004E005260B482430FEF70CFEED
:1078A000094820213830F9F717FE0748FF22F42154
:1078B0005C30F9F70AFEC4F8488030462763BDE81B
:1078C000F0870000C8810020108000204859002067
:1078D000496E76616C69646174696E67206F6C646F
:1078E000206170706C69636174696F6E20696E20CD
:1078F00062616E6B20302E002DE9F04104004FF0E4
:10790000010503D140497F20FBF7FCFD94F85400AA
:107910003E4E012740B194F8550050B1012808D0DF
:10792000022806D0032804D0308839A107EB004094
:1079300064E01CB934496720FBF7E4FD94F86D005E
:10794000032807D0308838A107EB004000F090FEF4
:10795000142556E094F88F00B84618B194F89000BA
:1079600000284ED1207A58B1E068022734280CD084
:10797000308832A107EB004000F07AFE112540E08C
:10798000318808EB014032A138E0204603F0AEF91F
:1079900018B1207850B394B907E0308830A107EBD4
:1079A000004000F065FE12252BE017498C20FBF704
:1079B000A9FD207818B914498D20FBF7A3FD94F890
:1079C00055002B4968B101280BD06068C96888420E
:1079D00017D8308827A107EB004000F049FE10259A
:1079E0000FE06068896888420BD2F2E794F855008E
:1079F000012806D0318808EB014023A100F038FEB1
:107A00000F252846BDE8F08180C30F004C590020A7
:107A1000496E76616C6964206669726D7761726522
:107A200020747970652E0000496E76616C6964205F
:107A30006861736820747970652E00004661756C0A
:107A400074792048572076657273696F6E2E000036
:107A50004E6F2048572076657273696F6E2E000056
:107A6000534420726571206E6F74206D65742E0012
:107A70001080002046572076657273696F6E2074FF
:107A80006F6F206C6F772E00465720766572736992
:107A90006F6E206D697373696E672E000FB438B511
:107AA000040003D110A11C20FBF72CFD606918B95C
:107AB0000DA11D20FBF726FD206818B90AA11E2084
:107AC000FBF720FD606818B907A11F20FBF71AFD1E
:107AD0000599002905D006A800906A46204600F0C6
:107AE00045F838BC5DF814FB2E2E5C2E2E5C2E2E35
:107AF0005C2E2E5C2E2E5C65787465726E616C5CFB
:107B0000667072696E74665C6E72665F66707269CA
:107B10006E74662E6300000010B5040003D107A147
:107B20000B20FBF7EFFCA268002A05D0D4E9040380
:107B3000216898470020A06010BD00002E2E5C2E0A
:107B40002E5C2E2E5C2E2E5C2E2E5C65787465725B
:107B50006E616C5C667072696E74665C6E72665F94
:107B6000667072696E74662E630000002DE9FC4732
:107B700091460C465FEA000804D183A14FF49F7040
:107B8000FBF7C0FCD8F8140020B97FA14FF4A07017
:107B9000FBF7B8FCD8F8000020B97BA140F24110F7
:107BA000FBF7B0FCD8F8040020B977A14FF4A1701E
:107BB000FBF7A8FC002C76D014F8011B39B125295D
:107BC0000ED04046FCF79EFB20780028F4D198F8B0
:107BD0000C00002867D04046BDE8FC47FFF79CBF7B
:107BE0000020012221782B291BD02D2902D03029F9
:107BF00008D102E040F0010001E040F00200641C06
:107C0000002AEFD100252A290ED02178A1F13002D7
:107C10000A2A11D205EB850201EB4205641C303DB6
:107C2000F1E740F00400EAE7D9F800100B1DC9F8AD
:107C300000300968641C0D44217800232E290BD1E3
:107C400014F8011FA1F130020A2A05D203EB8302C6
:107C500001EB4203303BF3E76C290DD068290BD0D0
:107C6000692921D00BDC252918D0582931D0632966
:107C70000ED0642915D117E014F8011FECE7702924
:107C800069D0732932D075291BD0782909D120E019
:107C9000D9F80000011DC9F8001001784046FCF732
:107CA00031FB641C90E76CE0D9F800100A1DC9F89C
:107CB00000200968CDE900500A224046FDF7AEFADF
:107CC000EFE7D9F800100A1DC9F8002009680A2258
:107CD00006E0D9F800100A1DC9F800200968102232
:107CE000CDE90050404603F00DFCDAE7D9F800106A
:107CF00000270A1DC9F800200E68C00705D112E050
:107D00004046761C7F1CFCF7FDFA31780029F7D13C
:107D100004E0202140466D1EFCF7F4FABD42C0D9B4
:107D2000002DF6D1BDE74EB13046F9F7E0FB07462E
:107D300004E0202140466D1EFCF7E4FABD4206D95E
:107D4000002DF6D103E04046761CFCF7DBFA3178D3
:107D50000029F8D1A5E7D9F80000011DC9F80010E5
:107D6000056830214046FCF7CDFA78214046FCF703
:107D7000C9FA08200021CDE9000103461022294656
:107D8000B0E7BDE8FC8700002E2E5C2E2E5C2E2E68
:107D90005C2E2E5C2E2E5C65787465726E616C5C58
:107DA000667072696E74665C6E72665F6670726928
:107DB0006E74665F666F726D61742E630000000002
:107DC0002DE9F0411E4615460F46040003D11DA1C2
:107DD0007820FBF797FB206818B91AA17920FBF7E8
:107DE00091FB1DB917A17A20FBF78CFB3946204681
:107DF000FBF72CF840B939462046FBF727F818B9AD
:107E000010A17D20FBF77EFB6068394602682046A2
:107E10006A43FBF724F858B960683946026820467F
:107E20006A43FBF71CF818B906A17F20FBF76AFB31
:107E3000206833462A46D0F810C039462046BDE8AF
:107E4000F04160472E2E5C2E2E5C2E2E5C2E2E5C7A
:107E50002E2E5C636F6D706F6E656E74735C6C69F3
:107E6000627261726965735C6673746F7261676573
:107E70005C6E72665F6673746F726167652E630015
:107E800070B516460C46050003D108A12F20FBF75C
:107E900039FB1CB905A13020FBF734FB2C603146BF
:107EA00028462268BDE87040104700002E2E5C2E48
:107EB0002E5C2E2E5C2E2E5C2E2E5C636F6D706FF2
:107EC0006E656E74735C6C69627261726965735C15
:107ED0006673746F726167655C6E72665F667374F9
:107EE0006F726167652E63002DE9F04128B101686A
:107EF00019B1C969BDE8F04108470D4D0D4800248E
:107F0000461B14270DE000BF04EB840005EB800046
:107F1000016829B1C969884710B10120BDE8F08125
:107F2000641CB6FBF7F0A042EED80020F6E7000094
:107F30001059002024590020044801214174007A7E
:107F400008B1002070470120704700007C870020A6
:107F5000012801D0032808D10449002201284A74CD
:107F600000D00020087402F03DBC70477C870020E0
:107F700070B50146022801D0032943D1224C207A52
:107F800000283FD0012831D002282FD11F480023DC
:107F90000229006802D0032928D119E0E3600279A0
:107FA00012B1012A22D10BE0D0E90565721B142A17
:107FB00000D314222A4482614569AA420ED015E0FA
:107FC0000169491C0161426991420FD1237213E09A
:107FD000E268521CE260082A08D9E3602372022991
:107FE0000AD00D21FCF7B9FE02F0F2FB607C28B14B
:107FF000BDE8704000F01EBF0021F3E7BDE870400F
:1080000002F0F0BB70BD00007C870020A05800206B
:108010002DE9F8431D46089F16468846040003D103
:108020002AA16220FBF76EFA1EB928A16320FBF794
:1080300069FA206818B925A16420FBF763FA1DB915
:1080400022A16520FBF75EFA60684068B5FBF0F19D
:1080500000FB115141B1B5FBF0F100FB115018B11B
:108060001AA16820FBF74EFA4046FAF7E9FE38B944
:108070004046FAF7E5FE18B914A16B20FBF742FA67
:108080003046FAF7DDFE38B93046FAF7D9FE18B9AE
:108090000EA16C20FBF736FA2A4641462046FAF735
:1080A000DEFE48B92A4641462046FAF7D8FE18B9FE
:1080B00006A16D20FBF726FA009720682B46324672
:1080C000C76841462046B847BDE8F8832E2E5C2E8F
:1080D0002E5C2E2E5C2E2E5C2E2E5C636F6D706FD0
:1080E0006E656E74735C6C69627261726965735CF3
:1080F0006673746F726167655C6E72665F667374D7
:108100006F726167652E63002DE9FF411C46DDE952
:108110000A7815460E46684600F010F846EA450112
:1081200041EA840141EA072242EA0841009A00EB51
:108130008200C0F80017BDE8FF81000010B50446BA
:108140000068302804D308A140F2A110FBF7DAF947
:108150002068202802D24FF0A04010BD00F01F0080
:1081600020600C4810BD00002E2E5C2E2E5C2E2EA2
:108170005C2E2E5C2E2E5C6D6F64756C65735C6E70
:108180007266785C68616C5C6E72665F6770696F5E
:108190002E6800000003005010B504460068302827
:1081A00004D308A140F2A110FBF7ACF92068202805
:1081B00002D24FF0A04010BD00F01F0020600C481C
:1081C00010BD00002E2E5C2E2E5C2E2E5C2E2E5C02
:1081D0002E2E5C6D6F64756C65735C6E7266785C78
:1081E00068616C5C6E72665F6770696F2E68000014
:1081F0000003005038B501240090684631B1FFF704
:108200009DFF00998C40C0F8084538BDFFF796FFE8
:1082100000998C40C0F80C4538BD000030B5104BBB
:10822000014600201C69224609E0157A854205D1E5
:10823000401C0A28F7DB4FF0FF3030BD5268002A9F
:10824000F3D1421CF9D008721A6922B152684A600F
:108250001A69516030BD002219614A6030BD0000CA
:10826000909800207047FAF70BBC704708B5034A96
:1082700000924023024A00F005F808BDBDAD0F0092
:1082800090870020F0B595B01C4615460F4608466D
:108290001A9E00F071FB182109A8F9F71DF90E9636
:1082A000CDE909540023082203A9384600F079FBE0
:1082B00005980690BDF81000ADF81C00BDF812003E
:1082C000ADF81E0000208DF821000398082600F06C
:1082D0000300012802D0022818D032E00398334668
:1082E000850AC0F3C2008DF8200003980FA9C0F3DF
:1082F0008314A200384600F054FB09A8009006AB96
:1083000022460FA9284600F093FA1AE00398840D3C
:10831000C0F3C2008DF82000082C01D2254600E0F1
:10832000082533462A460FA9384600F03AFB2E446A
:10833000641B09AB06AA29460FA800F0CDF9002C52
:10834000EAD1384600F01EFB15B0F0BD0A4A0129FB
:1083500002EBC00007D0022907D0032907D0042967
:1083600007D0002070470220704704207047007932
:108370007047407970470000B8CE0F0010B5FFF786
:1083800072FF04210648FFF749FF002803DA054978
:108390001B20FBF7B7F802490120487210BD00000E
:1083A000AC580020DCC80F002DE9F04F8DB0FBF772
:1083B000B9FF18B100200DB0BDE8F08F794E002054
:1083C000B061BFF34F8FA6F580544FF0000960688D
:1083D0000190A568284004EB800008E0216801981E
:1083E000814201D86160E5E7284004EB80000C3051
:1083F00001A9FCF767FF0028F0D105AAA046019962
:1084000001EA050408EB8403491CDB6842F82030CC
:10841000401C01910228F2D3059800F003000228C5
:1084200002D001284CD0A6E005985022810D8A4642
:10843000B2EB905F00D850210C4664F39F5005903A
:108440000831594800F04FFA070075D000F094FA4F
:108450004B46082205A9384600F0A9FA019909F10E
:10846000080B2940681A8000001D844221D94F4D15
:1084700030B1C2B208EB8101201A91460C3104E000
:108480002946E2B2002591462846C4B25B463846EA
:1084900000F08DFA0BEB090325B122462946384638
:1084A00000F085FA01990AF1030001EB90000190B8
:1084B0003BE008EB81015B46224638460C31EFE792
:1084C0000598C0F38310062800D30620059960F3B1
:1084D0008911C1F38310801C05918100324800F09E
:1084E00002FA070047D000F047FA4B46082205A9D8
:1084F000384600F05CFA09F1080900240FE0019801
:108500004B4600EA0501401C08EB81010190042262
:1085100038460C3100F04BFA09F10409641C059847
:10852000C0F38310A042EAD837B13469B06968B1AA
:10853000384600F027FA2FE01DE0607A012804D1C8
:10854000226820463946126890476468002CF4D1AE
:10855000384600F017FA00208DF800006846FAF758
:1085600041FFB06910B90199C8F804109DF80000E6
:10857000FAF784FF10E0346904E021682046896836
:1085800088476468002CF8D109480221008801EB73
:10859000004008A100F06CF8FBF7C4FE80F0010079
:1085A00009E700009098002080CF0F009C880020F1
:1085B0006C5900204261636B656E647320666C7554
:1085C00073686564000000002DE9F84F8146264F6E
:1085D000D01C15468A46800800226946BE68FBF713
:1085E0003BFEB8B3009CB846A01C0090B968304070
:1085F000091A8F003F1DBD4208EB800002D82A46B1
:10860000514608E03A4651460C30F8F73DFF16480F
:10861000EA1B0AEB07010C30F8F736FF4FEA19475F
:10862000FCF78EF947EA0042601C304008EB8000FE
:10863000344008EB8401C260C8684FF6C07269F329
:10864000C500904365F39F5020F00300801C20F08C
:108650000400C860054890F8200001E0FFF7A4FE80
:108660000028FBD1BDE8F88F90880020909800206A
:1086700000231A4602F07CBD08B5012300926A4629
:1086800002F076FD08BD1CB5CDE9002302236A4641
:1086900002F06EFD1CBD3EB5069C8DE81C00032358
:1086A0006A4602F065FD3EBD7FB5DDE908458DE80F
:1086B0003C0004236A4602F05BFD7FBD70B586B0C6
:1086C0000DF1280C9CE870008DE87C0005236A46BB
:1086D00002F04EFD06B070BD2DE9F0470E46804613
:1086E0001C46924608293ED894F80C90002020732E
:1086F0001946104602F012F80025B54206D218F8C5
:1087000005201AA12046FFF7C9F903E019A1204668
:10871000FFF7C4F96D1C082DEFD317A12046FFF712
:10872000BDF90025B54210D218F80570F8F7A8FE7B
:108730000068C05D10F03E0F01D03A4600E02E22E6
:108740000EA12046FFF7AAF903E00DA12046FFF78E
:10875000A5F96D1C082DE5D301222146504601F0F4
:108760005DFF84F80C90BDE8F087000020253032D2
:1087700078000000202020007C000000256300001D
:1087800020000000104910B540F2FF308860002042
:108790000860486001F580518861486181F82000D7
:1087A0000A4800F0EDF800280CD1094809490A4BA5
:1087B000401AC108002002E023F82000401C884233
:1087C000FAD3002010BD00009088002080CF0F0059
:1087D00068CF0F00B8CE0F0024590020024803498B
:1087E000401AC0087047000068CF0F00B8CE0F00D5
:1087F00013B56846FCF704FF08B100201CBD024811
:10880000009950F831001CBDB8CE0F0070B5074874
:108810000125046980F8205005E065722168204632
:10882000496888476468002CF7D170BD9098002093
:108830002DE9FF4781460C9D00200C462F7B2873B5
:10884000984616462946184601F068FF072E42D280
:10885000DFE806F004090F161F2A360049462846AD
:10886000FFF71CF937E0494628462268FFF716F95A
:1088700031E0D4E9002349462846FFF70FF92AE002
:10888000A0680090D4E9002349462846FFF706F97E
:1088900021E0D4E90201CDE90001D4E900234946F1
:1088A0002846FFF7FBF816E004F1080007C88DE83A
:1088B0000700D4E9002349462846FFF7EFF80AE00D
:1088C00004F108000FC88DE80F00D4E900234946E1
:1088D0002846FFF7E3F800222946404601F09EFEB5
:1088E0002F73BDE8FF872DE9F041858A80462D1F53
:1088F0004819C01CB0FBF5F0C6B24046FCF712FFA9
:10890000041E19D00020207101206071E58000272D
:108910002546761EC4F800800BE04046FCF702FFB7
:1089200060B16179491C6171286005467F1CC0F8FF
:108930000080B742F1D32046BDE8F081204600F028
:1089400002F80020F8E72DE9F041457901466B1E59
:10895000002201E00968521C9A42FBD30F680146CD
:10896000002605E038460C68FCF742FF2146761CDD
:10897000AE42F7D3BDE8F0810121001DFCF7ABBE8C
:10898000FCF77EBF10B504460121001DFCF7C4FEB4
:1089900010F0FF0F04D12046BDE81040FFF7D3BF11
:1089A00010BD38B501240094FCF7E0FD38BD38B5A2
:1089B00000240094FCF7DAFD38BD000009490222CA
:1089C0000A60BFF36F8FBFF34F8F0A1D1060064818
:1089D0000268002AFCD000200860BFF36F8FBFF34D
:1089E0004F8F704704E5014000E4014070B50E4C24
:1089F00001232360BFF36F8FBFF34F8F00230B4D15
:108A000008E000BF51F8236040F823602E68002E74
:108A1000FCD05B1C9342F5D300202060BFF36F8F26
:108A2000BFF34F8F70BD000004E5014000E401403A
:108A300020B1034909680160002070470E2070478B
:108A4000B0BD0F002DE9FE4307460D460846FFF76F
:108A5000EFFF00287ED18046CDF80080CDF804805D
:108A6000012406208DF80070ADF80400CDF80880D0
:108A70008DF80240694620202A6869DF3F4E40B1E8
:108A800000F0A2FB024630883D4904EB0040FFF7AE
:108A9000F3FDCDF800808DF801408DF80280CDF80F
:108AA0000480CDF808808DF80380694640202A684C
:108AB00069DF40B100F088FB02463088314904EBA1
:108AC0000040FFF7D9FDCDF800808DF80070F72049
:108AD000ADF80200CDF80480CDF808806946232067
:108AE0002A6869DF40B100F06FFB024630882649F2
:108AF00004EB0040FFF7C0FDCDF80080CDF8048006
:108B0000CDF808808DF800404746694601202A6864
:108B100069DF40B100F058FB024630881B4904EB86
:108B20000040FFF7A9FD4FF4B06000900197029755
:108B30006946A1202A6869DF40B100F045FB024682
:108B40003088134904EB0040FFF796FD009701972A
:108B5000029700E010E08DF800406946A0202A68E6
:108B600069DF40B100F030FB02463088094904EB70
:108B70000040FFF781FD0020BDE8FE83745900200E
:108B80002CCB0F0074CB0F00C0CB0F008CCA0F0092
:108B9000D8CA0F0038CA0F002DE9F0410446D0F8BA
:108BA000008060DF2168194D074641451CD928889F
:108BB000022606EB004016A1FFF75AFD2888424620
:108BC00006EB00401EA12368FFF75DFDF006D0F81C
:108BD0000C012168800200F10050421A288825A16A
:108BE00006EB0040FFF748FD012467B1384600F06E
:108BF000EBFA024628882AA104EB0040FFF73CFD6F
:108C00003846BDE8F0812E480470F9E77459002019
:108C1000496E73756666696369656E742052414D6D
:108C200020616C6C6F636174656420666F72207480
:108C3000686520536F66744465766963652E00002D
:108C40004368616E6765207468652052414D2073EA
:108C500074617274206C6F636174696F6E206672E8
:108C60006F6D203078257820746F20307825782E2D
:108C7000000000004D6178696D756D2052414D20F6
:108C800073697A6520666F72206170706C696361C8
:108C900074696F6E20697320307825782E0000008B
:108CA00073645F626C655F656E61626C6528292024
:108CB00072657475726E65642025732E0000000065
:108CC0000B59002030B51848ADF5017D007800281B
:108CD00026D04FF4FA7400BFADF8004280A9684670
:108CE00061DF38B105281BD00DF5017DBDE83040AE
:108CF000FAF756BA6D460D497DA800F0F1F809E083
:108D00007DA800F0D5F8D0E90021284690477DA83D
:108D100000F024F97DA800F0CBF80028DCD0EFE7C4
:108D20000DF5017D30BD00000B590020B4BD0F00D2
:108D3000F8B5134C2078C0B10120A07002F008F8FB
:108D4000112814D0022002F01FF800258DF80050E1
:108D50006846FAF747FB11DF064625709DF80000CC
:108D6000FAF78CFB2EB13046F8BD0820F8BD002084
:108D7000F8BDA57002F0A8F9032002F005F8F6E7A7
:108D8000085900207CB5194C207808B108207CBD1A
:108D90000120A070002001F0DBFF112819D0002075
:108DA00001F0F2FF12480026006801908DF8006083
:108DB0006846FAF717FB0F4901A810DF05000AD033
:108DC000002020709DF80000FAF758FB2DB12846CE
:108DD0007CBD00207CBD0120F3E7A670667002F028
:108DE0008FF9012001F0D0FFF3E7000008590020BF
:108DF00048BD0F0045310F000EB50A49684600F026
:108E00006FF808E0684600F047F8D0E9001088479E
:108E1000684600F0A3F8684600F03EF80028F1D15B
:108E20000EBD000064BD0F000148007870470000CF
:108E3000085900200548817819B1007818B1FFF76A
:108E400077BF08207047FFF79DBF0000085900203A
:108E50001FB568464BDF30B1052819D004B0BDE816
:108E60001040FAF79DB90B4901A800F039F809E064
:108E700001A800F029F8D0E900210098904701A846
:108E800000F06CF801A800F01FF80028E1D0EFE72F
:108E90001FBD0000D0BD0F0010B5040003D1034971
:108EA0009E20FAF72FFBA06810BD0000E4C90F0058
:108EB00010B5040003D103499E20FAF723FBA068F4
:108EC00010BD0000E4C90F0010B5040003D1034930
:108ED0009E20FAF717FBA06810BD0000E4C90F0040
:108EE00070B50D46040003D108492A20FAF70AFBA1
:108EF0001DB906492B20FAF705FB2560286860603C
:108F00002046BDE8704000F003B800009CC40F008C
:108F100010B5040003D110490D20FAF7F3FA2068C8
:108F200018B90D490E20FAF7EDFA606818B90A4928
:108F30000F20FAF7E7FAD4E900104A68904201D10D
:108F4000002004E0D0E900239A4202D01046A0603D
:108F500010BD08306060F0E79CC40F0010B504003D
:108F600003D112493D20FAF7CDFA206818B90F490C
:108F70003E20FAF7C7FAA068002815D02168896852
:108F80000844A060606818B908494D20FAF7BAFA99
:108F9000D4E901014268914206D108306060204660
:108FA000BDE81040FFF7B4BF10BD00009CC40F0027
:108FB00070B50D46060003D10BA11420FAF7A2FAF2
:108FC0001DB909A11520FAF79DFA746804E0B2688A
:108FD0002946904718B1246820680028F7D12068F6
:108FE0002860256070BD00002E2E5C2E2E5C2E2E7B
:108FF0005C2E2E5C2E2E5C636F6D706F6E656E74D2
:10900000735C6C69627261726965735C736F7274B0
:109010006C6973745C6E72665F736F72746C697383
:10902000742E630010B5040003D103A13D20FAF7AC
:1090300069FA206810BD00002E2E5C2E2E5C2E2EAC
:109040005C2E2E5C2E2E5C636F6D706F6E656E7481
:10905000735C6C69627261726965735C736F727460
:109060006C6973745C6E72665F736F72746C697333
:10907000742E630010B5040003D103A13720FAF762
:1090800041FA6068006810BD2E2E5C2E2E5C2E2EDC
:109090005C2E2E5C2E2E5C636F6D706F6E656E7431
:1090A000735C6C69627261726965735C736F727410
:1090B0006C6973745C6E72665F736F72746C6973E3
:1090C000742E630010B5040003D105A12B20FAF71C
:1090D00019FA61680868002801D002680A6010BDAA
:1090E0002E2E5C2E2E5C2E2E5C2E2E5C2E2E5C6385
:1090F0006F6D706F6E656E74735C6C6962726172B5
:109100006965735C736F72746C6973745C6E72669C
:109110005F736F72746C6973742E630070B50C4664
:10912000050003D10BA14320FAF7ECF91CB909A102
:109130004420FAF7E7F90021686806E0A24203D16B
:1091400021680160012103E010460268002AF5D180
:10915000084670BD2E2E5C2E2E5C2E2E5C2E2E5CB4
:109160002E2E5C636F6D706F6E656E74735C6C69D0
:10917000627261726965735C736F72746C69737427
:109180005C6E72665F736F72746C6973742E6300C9
:109190000C4A10B502F594730EE0991AC91001EB50
:1091A000D171491002EBC1010C68844201D90B4610
:1091B00002E005D201F108029A42EED3002010BD70
:1091C000486810BDF8BB0F0000B5FFF7E1FF0028AD
:1091D00000D1014800BD0000E4BB0F002DE9F041C3
:1091E00004461348134BC01A0C21B0FBF1F6A069DA
:1091F0004FF0FF3110F8022C02B92169002011E074
:1092000000EB400503EB85052F68974209D14F1C01
:1092100002D06F688F4204D194E80F00AD68A84770
:1092200003E0401CB042EBD301202060BDE8F08198
:10923000D4CF0F00C8CF0F0002480068002800D02C
:10924000012070470004014070B50C46050003D1B1
:109250000D49D920FAF756F91CB90B49DA20FAF76B
:1092600051F90A480421008801EB004008A1FFF7EA
:10927000FFF912490320C96888476869FEF722FA96
:10928000FBF7C0FD607070BD60C10F003C5900204D
:1092900048616E646C65204E52465F4446555F4F90
:1092A000505F4F424A4543545F4352454154452025
:1092B00028636F6D6D616E642900000028580020DE
:1092C00070B50C4620B9154940F20110FAF71AF9A9
:1092D00024B912494FF48170FAF714F9104D04269D
:1092E00010A1288806EB0040FFF7C2F91849081FB3
:1092F000FEF706FAFBF786FD6070012805D1002015
:10930000FEF702F810B10A20607070BD288811A124
:1093100006EB0040BDE87040FFF7AAB960C10F003E
:109320003C59002048616E646C65204E52465F4493
:1093300046555F4F505F4F424A4543545F4558453D
:10934000435554452028636F6D6D616E642900009C
:109350003058002057726974696E672076616C69B5
:109360006420696E697420636F6D6D616E64207432
:109370006F20666C6173682E0000000070B50D46AA
:10938000040003D11749E720FAF7BCF8206918B99F
:109390001449E820FAF7B6F8A08A18B91149E9206B
:1093A000FAF7B0F81DB90F49EA20FAF7ABF80E4802
:1093B0000421008801EB00400CA1FFF759F9A18AB4
:1093C0002069FEF73FF9FBF71DFD68702846FBF7A3
:1093D0008BF8E168002903D02069BDE87040084798
:1093E00070BD000060C10F003C59002048616E64F0
:1093F0006C65204E52465F4446555F4F505F4F426A
:109400004A4543545F57524954452028636F6D6D58
:10941000616E64290000000030B587B00C46054637
:10942000182218496846F8F72FF8207B0195164D49
:109430008DF80000012806D0022812D006281CD181
:10944000607B049019E01148FEF714F8A888E880C2
:10945000607B0490617CD4F80E0061F31F6005907E
:109460000BE00B480421008801EB004009A1FFF745
:10947000FFF8B4F80D00A880E8806846FDF7B4FC5A
:1094800007B030BD68BA0F0008580020B0CE0F00FA
:1094900030590020536574207265636569707420CB
:1094A0006E6F7469660000002DE9F0410B4E0D46A9
:1094B000042730880AA107EB0040FFF7D9F8114CC8
:1094C000308811A107EB0040A36C226DFFF7DBF899
:1094D000A06CA860206D6860BDE8F0813C59002058
:1094E00048616E646C65204E52465F4446555F4F3E
:1094F000505F4352435F474554202864617461299B
:1095000000000000108000204F66667365743A25E5
:10951000642C204352433A307825303878000000DC
:109520002DE9F84F3E4C81460D462088042707EB75
:1095300000403CA1FFF79CF8FEF76CF901264FF0C4
:10954000080AC8B1D9F814204FF00308DAB13F492E
:109550003F4813051CD0436DD1F808C01344634540
:1095600016D020883BA106EB004000BFFFF780F833
:1095700085F80180BDE8F88F20883FA106EB004008
:10958000FFF776F81EE0208849A106EB0040EDE7E2
:10959000B2F5805F07D920884CA106EB0040FFF7A9
:1095A00067F86F70E6E7436DD1F808C003EB020877
:1095B000E0450AD9CDF800C020884D4906EB0040AF
:1095C000FFF769F885F801A0D4E74264C26C03652F
:1095D000036380468264D9F81400002200F6FF700D
:1095E0004FEA103C486861461844FDF7F3F940B172
:1095F000208840A106EB0040FFF73AF8052068708C
:10960000B8E7D8F848100091208840A107EB004047
:10961000D8F85030D8F84420FFF73DF8AAE700000A
:109620003C59002048616E646C65204E52465F4490
:1096300046555F4F505F4F424A4543545F43524542
:109640004154452028646174612900002858002095
:10965000108000204F626A6563742073697A652008
:109660006D757374206265207061676520616C6937
:10967000676E65640000000043616E6E6F74206366
:1096800072656174652064617461206F626A6563EC
:109690007420776974686F75742076616C696420D2
:1096A000696E697420636F6D6D616E640000000007
:1096B0004F626A6563742073697A652063616E6EB8
:1096C0006F7420626520302E00000000496E7661C4
:1096D0006C69642073697A6520666F72206F626AB4
:1096E0006563742028746F6F206C61726765290050
:1096F000ECC00F004572617365206F706572617414
:10970000696F6E206661696C656400004372656113
:1097100074696E67206F626A656374207769746824
:109720002073697A653A2025642E204F666673653A
:10973000743A203078253038782C204352433A2030
:1097400030782530387800002DE9F041154D074676
:109750000E462888042101EB004013A1FEF788FF84
:109760001B4CD4E91401626C431A9A420BD028882E
:10977000012101EB004017A1FEF785FF0820707062
:109780000120BDE8F08100216164A16CE1646065A5
:109790000021384600F032F817490420C96888478C
:1097A0000020EEE73C59002048616E646C65204E55
:1097B00052465F4446555F4F505F4F424A454354BF
:1097C0005F4558454355544520286461746129001C
:1097D00010800020496E76616C6964206461746158
:1097E0002E2065787065637465643A2025642C20AA
:1097F000676F743A20256400285800202DE9F04155
:10980000044686B00020FEF76FFB224E012758B1B8
:10981000214A18212046F9F7DFFC020036D03088B3
:109820001EA107EB00402FE0182227496846F7F7F2
:109830002BFE2648264D4FF00408006DA96888428B
:1098400011D1318808EB014022A1FEF711FFD5E9C3
:109850000101FDF7E5FF8DF80100FBF7D3FA8DF864
:109860000100254D02E08DF801700025D4E90112B8
:109870006846904715B12846FDF746FD31889DF8AA
:10988000012008EB01401DA1FEF7F6FE06B0BDE881
:10989000F08100003C590020FD970F004661696C83
:1098A000656420746F207363686564756C65206FF0
:1098B000626A65637420657865637574653A203003
:1098C0007825782E0000000028BB0F0010800020B3
:1098D00028580020506F737476616C6964617469F4
:1098E0006F6E206F66206669726D776172652069A0
:1098F0006D6167652E000000A59A0F0052657175B5
:109900006573742068616E646C696E6720636F6D47
:10991000706C6574652E20526573756C743A2030D6
:1099200078257800F8B50C4D0C46042628880BA144
:1099300006EB0040FEF79CFE124813A1826CA26069
:10994000036DB0026360E0600090288806EB004081
:10995000FEF7A1FEF8BD00003C59002048616E648E
:109960006C65204E52465F4446555F4F505F4F42F4
:109970004A4543545F53454C454354202864617421
:109980006129000010800020637263203D20307840
:1099900025782C206F6666736574203D203078250D
:1099A000782C206D61785F73697A65203D2030786E
:1099B000257800002DE9F041264F05460E463888EF
:1099C000042101EB004024A1FEF752FEFDF722FF27
:1099D00098B12B4CD4E91401401AA98A0844616C4F
:1099E00088420CD93888012101EB004025A1FEF7FF
:1099F0003FFE03207070BDE8F0810820FAE7274998
:109A0000206B49684718E86820B925494FF4E07091
:109A1000F9F778FDD5E90331AA8A3846FDF78AF8C7
:109A200020B1D5E90310BDE8F0410847A98A206BB1
:109A3000134A08442063A98A206D483208442065EF
:109A4000A98A2869FAF76AFDA064B060206D706089
:109A5000D1E700003C59002048616E646C65204EDF
:109A600052465F4446555F4F505F4F424A4543540C
:109A70005F575249544520286461746129000000F1
:109A80001080002057726974652072657175657366
:109A90007420746F6F206C6F6E6700002858002070
:109AA00060C10F00074810B50088042101EB004099
:109AB00005A1FEF7DDFD11490620C968BDE810408B
:109AC000084700003C590020416C6C20666C6173B3
:109AD00068206F7065726174696F6E73206861765B
:109AE0006520636F6D706C657465642E2044465507
:109AF00020636F6D706C657465642E0028580020BB
:109B0000FEF784FEFEF750FC0028FBD10D4E6425C5
:109B10004FF47A47741C3846A0476D1EFAD10A48A4
:109B20000068C00700D000BEBFF34F8F0648E4387E
:109B30000168064A01F4E06111430160BFF34F8FF1
:109B400000BFFDE780B80F00F0ED00E00400FA056B
:109B500010B50446074804212246008801EB004066
:109B600005A1FEF789FD2146BDE810400748FBF737
:109B70003FBE00003059002046726565696E67205F
:109B800062756666657220257000000068CF0F0060
:109B90002DE9F0472F4F05464FF0040938880C4651
:109BA0004E4609EB00402CA1FEF762FD38882A7C66
:109BB00006EB004031A1FEF75FFD4FF44051374BFB
:109BC0004A6801204FF002089A4200D10220344E28
:109BD000326A012A00D1401C4FF0010C84F801C008
:109BE0002A7C1AB10025012A09D01BE084F80480E0
:109BF000F068A0602B48E060C0F57E200FE0D1F84F
:109C0000048098450ED125710878142801D9486937
:109C100000E00020A0604FF48050E0608868206180
:109C2000BDE8F087824208D284F804C0B068A06022
:109C3000FCF71CFCE060B069F1E7398809EB0140F2
:109C400019A1FEF715FDFF202071A560E5602561D3
:109C5000E6E700003C59002048616E646C65204EC8
:109C600052465F4446555F4F505F4649524D5741FB
:109C700052455F56455253494F4E00004669726D3A
:109C80007761726520696D616765207265717565C0
:109C9000737465643A20256400000000DBE5B1516F
:109CA0001080002000100F004E6F20737563682035
:109CB0006669726D7761726520696D616765000024
:109CC00030B58A1D8B79083187B0022B33D1538888
:109CD0008489A3422FD1127A012A2CD1184C0DF17C
:109CE000040C3CCC8CE83C000A89ADF80C204A8975
:109CF0000C3104911249ADF80E208039114C096ADB
:109D00000591CDF818D0018A05AA6088ADDF18B991
:109D10006846FAF76FF938B10020ADF8080001A9DC
:109D20006088B0DF50B106E040F2FD10ADF80800E9
:109D300001A96088B0DF002007B030BD0120FBE73B
:109D400080BA0F000858002070B506468C1DC888E0
:109D5000B18888B0884229D11948FBF7E3FC050097
:109D6000184825D0F42100910088042101EB00401F
:109D700063892A4614A1FEF78EFC628904F10C0166
:109D80002846F7F781FB1822174901A8F7F77CFB53
:109D9000029605956089ADF8180001A8FDF724F832
:109DA000002803D029460648FBF722FD08B070BD05
:109DB0000088022101EB00400CA1FEF759FCF5E7F9
:109DC00068CF0F0030590020427566666572202505
:109DD000702061637175697265642C206C656E20FA
:109DE000256420282564290090BA0F0063616E6EF7
:109DF0006F7420616C6C6F63617465206D656D6F4D
:109E0000727920627566666572210000F8B50D46AC
:109E100014460646694600F052FA00280ED0009A11
:109E2000FF2A0AD8501C824207D869780223B3EB74
:109E3000911F02D02979814201D20020F8BD227001
:109E4000611C304600F080FBF8BD114600F0D6B82A
:109E5000114600F0E3B8F8B50C46154606466946CB
:109E600000F02DFA00280CD0009A501C904207D325
:109E700061780223B3EB911F02D02179814201D294
:109E80000020F8BD2946304600F05EFB009A002114
:109E9000A954F8BD2DE9FF410C468E6817460546CA
:109EA000694600F023FB00280ED0A06800280BD0E4
:109EB00060783A46C0F3011002283146684606D061
:109EC00000F0DAF80199696004B0BDE8F08100F0B3
:109ED00086F8F7E77CB50D461446694600F08FF921
:109EE000002820D02879082806D0042809D0022884
:109EF0000AD001280CD015E0DDE90001C4E9000119
:109F00000AE00098206006E0009800B2208002E09D
:109F1000009840B22070C117DDE90023504059403D
:109F2000084301D000207CBD01207CBD7CB50D46DE
:109F30001446694600F09EF9002820D028790828A8
:109F400007D00021042809D002280AD001280CD00B
:109F500014E0DDE90001C4E9000109E00098206097
:109F600006E0009880B2208002E00098C0B2207025
:109F7000DDE9002350405940084301D000207CBD5A
:109F800001207CBD7CB50D461446694600F072F98F
:109F9000002821D02979082908D00098C21704295F
:109FA0000BD002290DD001290ED014E0DDE900020A
:109FB000C4E900020146134609E0C31701462060C8
:109FC00005E001B2218001E041B22170CB17414090
:109FD0005340194301D000207CBD01207CBD70B5E9
:109FE0000D46064614461146284600F09AFA2246C7
:109FF00029463046BDE8704000F03EB838B50C4602
:10A000000422694600F0A0FA002806D09DF803104B
:10A01000009861F31F602060012038BD1CB50C461C
:10A020000822694600F090FA002824D09DF801101B
:10A030009DF800209DF80230080E42EA012242EA13
:10A04000034240EA13409DF803309DF8041040EAB3
:10A05000132008439DF8051042EA036240EA0120FC
:10A060009DF8061040EA01409DF8071040EA0160A3
:10A07000C4E9002001201CBD2DE9F04F04469DB02D
:10A0800000200090064601904FF0FF3A0AA800F029
:10A0900069F94FF0010BE94682E012AB05AA06A967
:10A0A000204600F0C9F850B10AA8059900F06BF9F4
:10A0B00060B10B98407810F0300F53D060E09DF8FD
:10A0C0004800002870D11DB0BDE8F08F0598B0425F
:10A0D00042D30B9D0AAE0B98407800F00F00082881
:10A0E00012D0304600F066F90B98A842F3D15646DC
:10A0F0000599B14230D3D4F8088009919DF8181021
:10A1000008910E990D6820E00B980678F0E7296811
:10A110000F682FB1DDE9083229462046B84711E023
:10A1200011948968DDE90872097891420CD12946B9
:10A1300017A8FBF76BF985F80CB017AA39461198E8
:10A14000FAF749FA0028BED0AD6815B1A1684145BB
:10A15000DDD0A168414523D19DF81810204600F0BC
:10A160002FFA1BE00C9840280AD200F01F010BFACE
:10A1700001F00C994A0959F82230034349F822307A
:10A18000E5682DB10AAB9DF8182020460599A8472F
:10A190000AAA9DF818102046FAF71DFA002892D056
:10A1A000A06800287FF479AFDDE90B0445780AA8A0
:10A1B00000F000F90028F7D115F0300F03D10B980B
:10A1C000007800B1641CC4B10020494605E000BF1E
:10A1D00051F82020521C0ED1401CB0EB541FF7D375
:10A1E000600959F8201004F01F00C0F120022AFA7B
:10A1F00002F0814201D0002065E7012063E71CB531
:10A200000C46694600F036F8002814D0DDE900025B
:10A21000C10709D051084FEA30006FEA00026FEA27
:10A220000100C4E9002004E051084FEA3000C4E90D
:10A2300000014FF001001CBDF8B507460020187062
:10A2400008700E4610601C4615466946384600F0F8
:10A2500036F8012140B1009850B1C10800F0070064
:10A26000296030700120F8BDB86808B10020F8BD41
:10A270002170FBE72DE9F8430026884681463446E5
:10A28000354604E0402E02D30020BDE8F88369463D
:10A29000484600F085F90028F7D09DF80070324656
:10A2A00007F07F00C10FF7F7DCF829430443F61DE0
:10A2B0000D463806E6D4C8E900410120E5E7F8B5C7
:10A2C0000E460746694600F06BF900280AD09DF853
:10A2D0000040200616D5072504F07F0403E0202D5A
:10A2E00001D30020F8BD6946384600F059F900282E
:10A2F000F8D09DF8001001F07F00A8400443ED1D48
:10A300000806ECD401203460F8BD000059680A4A00
:10A31000896891420ED1D0E901120848491C521EA9
:10A32000C0E9011206480421008801EB004005A1A4
:10A33000FEF7A2B9704700000CB90F003858002092
:10A340004859002050423A20496E69742070616378
:10A350006B65742064617461206C656E3A202564BD
:10A3600000000000C26000230160C0E901138B7887
:10A370001A44026191F903301A44426108780028B6
:10A3800000D00120704770B545680E4604466068ED
:10A390000178B14206D1407800F00F00082801D0C2
:10A3A000012070BD204600F005F86068A842EED19B
:10A3B000002070BD30B541680A785AB101F10C0334
:10A3C00043600A7B42B14C780A79C4F30115032D2E
:10A3D00007D00BE0002030BDC2680168FFF7C2FF64
:10A3E000F8E75D78C5F30115032D07D00225B5EB1D
:10A3F000141F09D14C7914FB02F209E08D7804692D
:10A400000022641B046103E0B5EB941F00D1042219
:10A41000497811F0300F02D18168491C81609C7825
:10A42000016921441144016193F903201144416100
:10A43000012030BD30B54168002487B0497801F073
:10A440000F02082A11D08A091ED00222B2EB911FF6
:10A4500009D10269C1F301110229146001D0032955
:10A4600001D14069047007B030BD0069056808E09B
:10A470002C7329466846FAF7C9FF6846FFF7DAFFEA
:10A48000AD68002DF4D1EEE7C1F30111012912D01E
:10A490000229E6D00329E4D04268517801F00F0187
:10A4A00007290BD0916881B11279006907B0BDE826
:10A4B0003040F6F7E9BF41690C70EDE7016990683B
:10A4C00007B0BDE8304000F02CB81179006907B042
:10A4D000BDE83040F7F700B810B5034B002408C0C2
:10A4E00080E8160010BD0000E9420F0038B50D46A7
:10A4F00004466946FFF7E3FE00280BD0D4E90002CA
:10A50000D4E90213C5E90002C5E9021300988142AB
:10A5100001D2002038BDA860A168081AA0600120FF
:10A5200038BD00B50A4687B001466846FFF71AFFF6
:10A53000002807D06846FFF77DFF6846FFF73AFF1F
:10A540000028F7D107B000BD7FB514460546A9B96C
:10A55000124A2868904208D110E010226946284625
:10A56000FFF7F2FF002807D0103C102CF5D8224648
:10A5700069462846FFF7E8FF04B070BDA868A0420E
:10A5800001D20020F8E72B68224628469847002889
:10A59000F2D0A868001BA8600120EDE7E9420F0097
:10A5A00010B504468068002809D02368012220469F
:10A5B0009847002803D0A068401EA060012010BD6D
:10A5C00038B5002439B1012912D0022912D0052949
:10A5D0001DD0002038BD0546012269462846FFF7F8
:10A5E000B3FF90B19DF800000006F5D4012038BDFE
:10A5F00008220DE005466946FFF761FE28B10021FB
:10A600002846009AFFF7A0FF38BD204638BD042237
:10A61000BDE838400021FFF797BF000010B50C4699
:10A62000017A052908D0407A38B1084808A10268A3
:10A630002046FDF733FA00E01AB106A12046FDF7E7
:10A640002DFA2046BDE81040FDF766BAE458002018
:10A65000257300000D0A00002DE9F047284D9946AA
:10A660001646044681B3284F09F50052DFF894C01E
:10A6700038885368A16D4FF0010808EB004063452E
:10A6800001D022490AE093684A1EC2F30B02891ADC
:10A6900041F6FF7211448B4205D21D49FDF7E8FFD8
:10A6A0000020BDE8F0874846FAF74AFE90B13888A6
:10A6B000022101EB00401749FDF7DAFF2EB11048E7
:10A6C0001830FBF7F9FE06E00CE0398808EB014092
:10A6D0001149E3E70EB1AC2000E0A520E862A06DCF
:10A6E000686301E0AA20E8623EB194F88F0010B1DF
:10A6F00094F8900008B96068E8600120D1E7000094
:10A7000010800020DBE5B15148590020A0C20F00A5
:10A7100034C20F00F4C20F00F0C10F0038B5C38877
:10A720000D46044633B114A0009015A216A1284688
:10A73000FDF7B4F9217A05291CD0607A48B1A088C8
:10A74000FDF704FE164951F8202016A12846FDF712
:10A75000A5F9A0880021FEF74BF803461049207A9E
:10A76000143951F8202001B02846BDE830400EA130
:10A77000FDF794B938BD00001B5B306D0000000090
:10A780001B5B313B33316D0025734C6F6773206465
:10A79000726F70706564202825642925730D0A0086
:10A7A000E4580020257300003C25733E2025733AB1
:10A7B00020000000EFF30580C005C00D01D001208E
:10A7C0007047EFF3148040F30000401C7047000016
:10A7D000034802490068FAF751BF0000A45800205E
:10A7E000B4BB0F002DE9F041224C0025224E207A07
:10A7F000012730B92148311D0068FAF74AFF30605F
:10A8000038B1022020723168087928B101281CD1A2
:10A8100014E06560BDE8F081D1E90503C01A142891
:10A8200000D31420B7EB900F01D2820800E0012280
:10A830000869C9681844194429DF03E0D1E9030114
:10A84000084428DF58B1112812D003213068FAF7E4
:10A8500084FA25726560BDE8F041FFF7B9BF207C3E
:10A860000028D7D1BDE8F04100210220FDF780BBD0
:10A870002772CFE77C870020A0580020B4BB0F00D0
:10A8800010B5074C201DFAF723FF002806D1607C85
:10A89000002803D1BDE81040FFF7A4BF10BD0000A1
:10A8A0007C87002010B510461A46F6F7EDFD002013
:10A8B00010BD10B510461A46F6F7E6FD002010BD93
:10A8C0002DE9F0411E681C461546074621B10129B5
:10A8D00018D0052923D119E000202060401C2060F9
:10A8E000B0421CD8012229463846FFF72DFE002829
:10A8F00006D015F8010B000601D52068EEE701200F
:10A90000BDE8F08108200246186002E004200246FB
:10A91000186029463846BDE8F041FFF715BE002013
:10A92000EEE770B516460A460446C11C104600F014
:10A93000C7FD054661193046C91C00F0C1FD284419
:10A9400070BD000003B5094A85B0D2E91612CDE901
:10A95000001207498989ADF8001006A9CDE9021057
:10A96000044869464088AEDF07B000BD00BA0F005A
:10A97000FC6D0020085800200846704708467047C4
:10A980002DE9F0418046FAF7C4F81A4D0026F0B1DF
:10A99000686828B168684068696820F07F4048604E
:10A9A00000F0DAFB040012D04FF080776068B84204
:10A9B00003D2204600F086FC03E0606820F07F4070
:10A9C00060602046FEF72EFB08B10446EEE700214A
:10A9D0004046F9F7BFFF28B1686818B1686800F011
:10A9E00071FC6E60404600F0D1FC4046BDE8F0418D
:10A9F00000F002B8545800202DE9F041214C0746E0
:10AA0000002600BF00F0A8FB90B341686068406872
:10AA100062685AB16268002A28D0884226D96068E4
:10AA2000007E18B161681848FEF7C2FA00F09AFB80
:10AA30004268054613484FF47A7300210830FAF74C
:10AA400089F830B10D2807D010499C20F8F75AFD3D
:10AA5000D8E7606820B106E0284600F033FCD1E773
:10AA60003846FAF75BF86560002ECBD1BDE8F0817F
:10AA7000FFE760680028F9D13846BDE8F041FAF7F1
:10AA80005BB800005458002060BB0F00CCC30F001F
:10AA90002DE9F05FFCF7EAFCDFF8CC80334D0427AA
:10AAA000D8F83020D8F8346000EB020BB01A411E01
:10AAB000C1F30B01401A00F6FF7A28882CA107EB9E
:10AAC0000040D8F84840FDF7D3FD42F20400324977
:10AAD00000594FF00109884208D0298809EB01404C
:10AAE0002EA1FDF7C5FD0320BDE8F09FD8F830008A
:10AAF0000444B04207D1288835A107EB0040FDF798
:10AB0000B7FD0020F0E7D0B904F500500178142912
:10AB100001D9406900E000203249B0FBF1F34FF465
:10AB200040500278142A01D9406900E00020B0FBAF
:10AB3000F1F228882CA107EB0040FDF7A4FD0823C3
:10AB4000524621465846FAF75DFA040007D0298894
:10AB500009EB01402FA1FDF78BFD2046C4E7BDE8BE
:10AB6000F05F0020FCF7D0BB108000206C59002063
:10AB7000456E746572206E72665F626F6F746C6F83
:10AB8000616465725F6466755F73645F636F6E7442
:10AB9000696E756500000000DBE5B151536F757299
:10ABA0006365206164647265737320646F657320EC
:10ABB0006E6F7420636F6E7461696E2061207661C0
:10ABC0006C696420536F66744465766963652E0012
:10ABD000534420616C726561647920636F706965AC
:10ABE0006400000040420F005570646174696E6734
:10ABF0002053442E204F6C64205344207665723AD3
:10AC00002025642C204E6577207665723A202564D5
:10AC1000000000004661696C656420746F20636FFA
:10AC20007079206669726D776172652E0000000090
:10AC300070B50F4C0421208801EB00400DA1FDF7F9
:10AC400017FDFFF725FF05004FF0010604D020880F
:10AC500010A106EB004007E0F8F760FC050006D005
:10AC6000208812A106EB0040FDF702FD284670BDCA
:10AC70006C590020456E746572206E72665F646662
:10AC8000755F73645F626C5F636F6E74696E756528
:10AC90000000000053442B424C3A20534420636F81
:10ACA0007079206661696C656400000053442B4232
:10ACB0004C3A20424C20636F7079206661696C6564
:10ACC0006400000070B50346002002464FF4405473
:10ACD00009E000BF53F82250A689B54201D10120F6
:10ACE00070BD521CD2B28A42F4D370BD10B50400BC
:10ACF00003D115493220F8F705FC4FF440501349B1
:10AD00004068884215D1217C04F1140009B16269C0
:10AD10004AB994F8552012B1012A08D10DE0012951
:10AD200005D962691AB9BDE81040FFF7CBBF012011
:10AD300010BD207C18B1606908B1002010BD2078DA
:10AD40000028F4D110BD000080C30F00DBE5B15135
:10AD50003EB504460B496846FEF7C2F80AE068466D
:10AD6000FEF79AF8D0E900212046904740B16846A6
:10AD7000FEF7F4F86846FEF78FF80028EFD13EBDE5
:10AD800011203EBD4CBD0F003EB504460A49684641
:10AD9000FEF7A6F809E06846FEF77EF8D0E9002144
:10ADA000204690476846FEF7D9F86846FEF774F8E3
:10ADB0000028F0D13EBD000058BD0F002DE9F04144
:10ADC0001400884618D000250E4F032608EB050115
:10ADD00022460020F7F756FE0544241A40B9387879
:10ADE000002809D008494FF47A408847761E05D0DC
:10ADF00001203870002CE9D1BDE8F08100203870C6
:10AE0000FAE70000A858002031BD0F0070B5184CBB
:10AE10000421208801EB004016A1FDF729FC1F4DFD
:10AE2000012308221C496888B1DF00281FD10223B2
:10AE3000002211466888B1DF002818D116484FF665
:10AE4000FF72083001886888AFDFA0F540510239F1
:10AE500003D0082801D0112809D12188022202EB51
:10AE6000014302460E491846FDF706FC002070BD5E
:10AE70003059002053656E64696E672053657276A1
:10AE8000696365204368616E67656420696E646903
:10AE9000636174696F6E0000F46D00200858002033
:10AEA00058C00F00FEB5474C2020029020880F4666
:10AEB0000325164605EB004043A1FDF7D9FB46B13B
:10AEC000208805EB00406FB149A1FDF7D1FB1620AA
:10AED000FEBD2088022101EB00404BA1FDF7C8FB1D
:10AEE0001320FEBD4D4F4EA1BA68FDF7C5FB02A968
:10AEF0005848CDE90001D7E901235749A0F58A70E8
:10AF0000FBF724F910B93278402A01D00A20FEBD9F
:10AF10005048711C4038F6F7B7FA20884FA105EB6E
:10AF20000040FDF7A5FB4B4840214038CDE900012A
:10AF3000A0F14801474AA0F5BC70029BFBF7CEF890
:10AF40000200208836D0012101EB004048A1FDF726
:10AF500093FB2088042505EB00404EA1FDF788FBFC
:10AF600020883C4905EB004040224039FDF72CFB8E
:10AF700020884BA105EB0040FDF77AFB029835498C
:10AF800082B2208805EB0040FDF71EFB208846A119
:10AF900005EB0040FDF76CFB2088402205EB0040EC
:10AFA0004449FDF711FB00BFFDF7FEF90028FBD176
:10AFB0000520FEBD05EB00403FA1FDF759FB012038
:10AFC000FEBD0000485900205369676E61747572B8
:10AFD000652072657175697265642E2043686563CA
:10AFE0006B696E67207369676E61747572652E0098
:10AFF000496E76616C6964207369676E61747572FD
:10B0000065207479706500004E6F207369676E610A
:10B010007475726520666F756E642E003858002056
:10B0200043616C63756C6174696E6720696E6974E5
:10B03000207061636B657420686173682028696E95
:10B040006974207061636B6574206C656E3A2025AD
:10B0500064290000FC840020CCB80F00566572699A
:10B060006679207369676E6174757265000000000F
:10B070005369676E6174757265206661696C656499
:10B0800020286572725F636F64653A203078257896
:10B09000290000005369676E61747572653A00009B
:10B0A000486173683A0000005075626C6963204B18
:10B0B00065793A003CB80F00496D61676520766597
:10B0C000726966696564000010B51620F7F7A6FE80
:10B0D00048B10A4882684FF4800152B1016821F4F6
:10B0E0008001016010BDBDE8104042F20100F8F798
:10B0F00057B84FF0E020C0F8801110BD94850020B3
:10B1000010B51620F7F78AFEA0B1114890F8000498
:10B110004009082811D280B101280ED004280CD093
:10B120000C4882684FF480016AB1016841F48001E3
:10B13000016010BD42F2010001E042F20200BDE8F0
:10B140001040F8F72DB84FF0E020C0F8001110BD06
:10B1500016E000E0948500200148FDF78BBF000059
:10B1600060BB0F000148FDF7ADBF000060BB0F00E2
:10B170002DE9F84FDFF89C809346894606461F4626
:10B18000012269461846D8F80850F9F765F8B0B3B7
:10B19000009800210446C246801C08E000EA05022F
:10B1A0005BF821300AEB8202401C491CD360B94293
:10B1B000F4D3C846B946370CF9F7C2FB8346FDF70E
:10B1C0000DFBB84204D8144940F28310F8F79AF9FD
:10B1D000601C28400AEB80002C4047EA0B420AEB37
:10B1E0008401C260C86866F3C50069F3891068F31A
:10B1F0009F2020F00300401C20F00400C860074896
:10B2000090F8200002E000BFFDF7CEF80028FBD147
:10B21000BDE8F88F9088002030C90F00909800207A
:10B220001FB5134800F15C01826B6846FFF754F9C3
:10B2300010489DE80E0080E80E000E490E48104AA6
:10B24000C8600E490020486088600E490948FEF732
:10B25000C6FE10B1012004B010BD0B4801210088CA
:10B2600001EB004009A1FDF703FA0020F3E700001D
:10B2700010800020648400200DA30F0038580020A7
:10B28000C8810020D8B90F004859002048616E6479
:10B290006C65723A20496E76616C69642070726FD9
:10B2A000746F636F6C20627566666572206D5F7087
:10B2B000625F73747265616D00000000002800D049
:10B2C0000047704770B50446C06818B90F4961203F
:10B2D000F8F718F90E4800250078A0B19CB1207E3F
:10B2E00088B1D4E903108847A06850B1217E41B1EC
:10B2F00061680844606021460648FDF759FE012553
:10B3000001E000202076284670BD0000CCC30F006D
:10B310005458002060BB0F0070B5164C20780028F0
:10B3200027D1154801680125C1F3004131B91349FE
:10B330000D600168C1F300410029FAD0F7F7F6FF6C
:10B3400008B1F7F72DFF0E4A00210E48F7F7D0FF9E
:10B3500018B10D492E20F8F7D5F80A48084A0121FE
:10B36000001DF7F7C5FF18B107493320F8F7CAF8F1
:10B37000257070BDF85700201804004008000040F8
:10B38000BDB20F00B8B80F0088BE0F002DE9F8431A
:10B39000244D814669462868FAF77BF90446002760
:10B3A0004FF00108204E39E0207820B101281BD051
:10B3B00002282AD122E06068017E31BB80F8188023
:10B3C0004846F9F7CEFA014660684268511A174AB2
:10B3D000914203D9416821F07F4141601148616881
:10B3E0000830FDF7E5FD10E061687068814200D12A
:10B3F00077600C480830FDF791FE06E0FFF7B2FEDB
:10B4000008B10776FAE786F8008069462868FAF7F7
:10B4100035F969462868FAF73CF90446002CC3D18F
:10B42000BDE8F88358BB0F005458002017FCFF00FC
:10B43000F8B50B4C0D46064669462068FAF713F935
:10B4400058B10670456069462068FAF72DF910B1C9
:10B450000448F9F74DFB0020F8BD0420F8BD0000BA
:10B4600058BB0F005C58002070B515460C460646C8
:10B47000FFF752FF3046F7F7A3FF18B10F494320FB
:10B48000F8F740F8002C17D0610CE0034FF4FA7283
:10B49000801841F1000152000023F5F7B1FF014689
:10B4A0002A463046F7F768FF002805D0BDE870400F
:10B4B00002494A20F8F726B870BD000088BE0F0088
:10B4C0000870020A4A70020C8A70000EC8700420CC
:10B4D0007047000010B50248FAF7F1F8002010BDDF
:10B4E0008858002010B514210448F5F7F5FF0448EA
:10B4F0000068FAF79DF8002010BD00007C8700204E
:10B50000B4BB0F002DE9F05F8346DDE90A4A994696
:10B5100090460D460846012703E000BFB0FBF8F057
:10B520007F1C4045FAD2B94500D94F465FEACA7040
:10B5300012D18CB15FEA8A7002D5B9F1000F01D047
:10B54000202607E0302605E031465846641EF8F70D
:10B55000D9FE0CB1A742F7D35FF00106B9F1010F94
:10B5600002D9A9F1010903E0B5FBF6F0404502D389
:10B5700006FB08F6F2E7DFF83C9000BFB5FBF6F0FB
:10B5800000FB165519F800105846F8F7BBFEB6FB3D
:10B59000F8F6002EF2D15FEACA7009D0002C07D06D
:10B5A000A74205D220215846641EF8F7ABFEF5E706
:10B5B000BDE8F09F76BB0F002DE9F041084601245D
:10B5C0001646254600212B460A46FAF77FFF0C4F08
:10B5D00038B138880BA105EB0040FDF749F8042489
:10B5E0000BE0FAF759FF30603988042202EB01437F
:10B5F00002460BA11846FDF73FF82046BDE8F08152
:10B600004859002043616E27742066696E64207279
:10B610006F6F6D20666F72207570646174650000D5
:10B620005772697465206164647265737320736511
:10B630007420746F20307825303878002DE9F0417F
:10B640000F24002790F85520184E01251AB990F8BC
:10B650006430012B06D0D30707D090F85630012B69
:10B6600002D002E0876E0DE0876D92070AD590F850
:10B670005C20012A06D1026E0D48C0F57E239A4255
:10B6800004D817444FB101240F600CE0308809A1A1
:10B6900005EB0040FCF7F7FF042430880DA105EB13
:10B6A0000040FCF7E5FF2046BDE8F0814859002046
:10B6B00000100F00424C2073697A65202825642908
:10B6C000206F766572206C696D6974202825642965
:10B6D00000000000496E6974207061636B6574201E
:10B6E000646F6573206E6F7420636F6E7461696E32
:10B6F0002076616C6964206669726D77617265207D
:10B7000073697A650000000030B10068054988421D
:10B7100005D048F20250704748F2015070470020AF
:10B72000704700006E52464870B5FDF785FD002851
:10B7300011D00020084A094B094C0121166801FA72
:10B7400000F52E4203D004EB8005C5F80036401CFE
:10B75000C0B20728F2D370BD080501403546526ECD
:10B7600000000140084810B5407800280BD0074879
:10B770000321008801EB004005A1FCF779FFBDE83B
:10B780001040FFF7D1BF10BDFA5700202C59002000
:10B79000496E7465726E616C2066656564000000B8
:10B7A00000207047002070472DE9FC4180461C4670
:10B7B00017460E460C48089DF9F78AFF10B1112074
:10B7C000BDE8FC81A20839463046FDF70FF906486E
:10B7D000F9F775FF33463A4601214046CDE9004569
:10B7E000F9F7A0FA0020EBE7885800202DE9F84F80
:10B7F000114D884681461E4617466946DDF828A049
:10B800002868F9F730FF040013D01C21F5F764FE17
:10B8100000202071C4F80090C4E90486C4E902A79E
:10B8200069462868F9F740FFFFF72AF80020BDE8CD
:10B83000F88F0420FBE70000B4BB0F0065FC2BF879
:10B8400016DA019ADE75D4A8477196211C875569CE
:10B85000105ABE04578FD2B0299456B8CA0363D683
:10B8600035C64DA7819FEFA7D2ECB7F307FF80AF96
:10B870007A3B4C19B891C5143CE8766D0000000085
:10B880000338FDD870470D0E0F100B0C181900006F
:10B890000338FDD8704700000000000000000000E1
:10B8A000000000000000000000000000FFFFFFFF9C
:10B8B0000000000000000001C0570020DC570020FD
:10B8C00048000000002040000000000031440F004C
:10B8D00041440F00DD430F00200000000000000085
:10B8E0000000000000000000010100000100000055
:10B8F0000000000002050000210000000000000020
:10B90000000000000000000000000000011104FC25
:10B910000400000000000000021104FC040000000C
:10B9200000000000032104FC0410000000000000DF
:10B93000041101FF0100000000000000051102FEDB
:10B940000400000000000000061104FC04000000D8
:10B9500000000000071104FC0400000000000000CB
:10B96000081701FF22000000E8B80F00091001FFCE
:10B9700001000000E4B80F0000000000000000001B
:10B9800000000000011101FF0100000000000000A4
:10B99000021702FE940000000CB90F000000000026
:10B9A00000000000000000000107000098000000F7
:10B9B00084B90F0002010000010000000000000037
:10B9C000030500004100000000000000000000002E
:10B9D0000000000000000000011704FC98000000B7
:10B9E00084B90F00021704FCDC000000A8B90F00A6
:10B9F0000000000000000000000000000000000047
:10BA000000210300002113000200000001000000DB
:10BA10000338FDD870470C000C00000058020000ED
:10BA20000200000000000000020000000000000012
:10BA30009C6D0020090000000000000000000000D4
:10BA400001000000000000002800000000000000CD
:10BA500000000000000100000000010000000000E4
:10BA600000000000000000000000000000000000D6
:10BA700039370F0000000000000000000000000047
:10BA800002000000000001000000000000000000B3
:10BA9000080000000000000039370F00519B0F0024
:10BAA0000000000000000000040000000000000092
:10BAB0000000000000000000000000000000000086
:10BAC0000000000000000000000000000000000076
:10BAD000F40000000000000018000000000000005A
:10BAE0000000000000000000000000000000000056
:10BAF0000000000000000000000000000000000046
:10BB0000170000000000000050EADA308883B89F78
:10BB1000604F15F30000C98E020000000000000015
:10BB20000000000000000000040000000000000011
:10BB30000000000000000000000000000000000005
:10BB400000010000000000000000000000000000F4
:10BB50000000000000000000645800200000070002
:10BB600000000000785800200D450F000000000084
:10BB70000338FDD8704730313233343536373839F1
:10BB8000414243444546000000100000040000000C
:10BB900001000000D9510F00D5B40F00A5A80F0077
:10BBA000A9B70F00914C0F0079A90F00A1B70F00A2
:10BBB00021530F008C5800200010000004000000EA
:10BBC00001000000E5510F00E5B40F00B3A80F001D
:10BBD000EDB70F00D94C0F007DA90F00A5B70F00DE
:10BBE00031530F00556E6B6E6F776E206572726FFA
:10BBF0007220636F646500000000000068C80F00D9
:10BC00000100000014C70F000200000008C50F006B
:10BC10000300000088C70F0004000000DCC70F000D
:10BC200005000000BCC60F000600000058C60F004B
:10BC300007000000C4C70F0008000000D0C60F00B6
:10BC40000900000034C70F000A00000050C80F00B0
:10BC50000B000000F0C40F000C000000E8C60F004D
:10BC60000D000000B8C80F000E000000B4C70F00A0
:10BC70000F000000F0C70F001000000024C80F00E4
:10BC800011000000CCC80F0012000000A0C80F0077
:10BC9000130000003CC80F008000000070C60F00B9
:10BCA00081000000ACC50F00820000006CC50F00D1
:10BCB000830000004CC50F008400000088C50F0001
:10BCC0008500000094C60F00860000009CC70F008E
:10BCD0009000000038C60F00910000002CC50F0036
:10BCE00092000000FCC60F000082000004C80F0094
:10BCF0000182000050C70F00028200006CC70F00D5
:10BD000000840000C8C50F000184000074C80F0043
:10BD10000284000010C60F0003840000ECC50F0071
:10BD20006D820F006B820F0065820F000000000023
:10BD30000338FDD870470000A0CF0F00A8CF0F0038
:10BD400000000000000000000100000738BD0F00E7
:10BD500048BD0F000800000070BD0F0080BD0F003F
:10BD60000800000080BD0F0090BD0F00080000001B
:10BD7000C0CF0F00C8CF0F0000000000000000007F
:10BD8000B0CF0F00C0CF0F00000000000000000087
:10BD900000000000000000000000000000000000A3
:10BDA00098CF0F00A0CF0F0000000000000000009F
:10BDB000B857002090BD0F00B0BD0F000800000074
:10BDC000A8CF0F00B0CF0F0000000000000000005F
:10BDD000C0BD0F00D0BD0F0008000000859F0F0000
:10BDE0002D9F0F00D59E0F004B9E0F00519E0F0000
:10BDF0000D9E0F00579E0F00959E0F000000000043
:10BE0000004040404040404040404141414141406D
:10BE10004040404040404040404040404040404022
:10BE200040050202020202020202020202020202B1
:10BE300002202020202020202020200202020202B6
:10BE4000020290909090909010101010101010100E
:10BE5000101010101010101010101010020202021A
:10BE6000020288888888888808080808080808085E
:10BE7000080808080808080808080808020202025A
:10BE80004000000001BE0F002E2E5C2E2E5C2E2ED8
:10BE90005C2E2E5C2E2E5C636F6D706F6E656E7403
:10BEA000735C6C69627261726965735C626F6F74F6
:10BEB0006C6F616465725C6E72665F626F6F746CEA
:10BEC0006F616465725F6466755F74696D657273D6
:10BED0002E6300002E2E5C2E2E5C2E2E5C2E2E5CF1
:10BEE0002E2E5C636F6D706F6E656E74735C6C6923
:10BEF000627261726965735C626F6F746C6F6164AA
:10BF000065725C6E72665F626F6F746C6F616465A0
:10BF1000725F66775F61637469766174696F6E2EB4
:10BF20006300000043524320636F6D707574617449
:10BF3000696F6E206661696C656420666F7220634C
:10BF40006F70696564206170703A2073726320635A
:10BF500072633A203078253038782C20726573204F
:10BF60006372633A20307825303878004120536F6F
:10BF7000667444657669636520686173206A7573C9
:10BF800074206265656E20616374697661746564AE
:10BF90002E2049742773206C696B656C7920746856
:10BFA000617420616E206170706C69636174696F87
:10BFB0006E2077696C6C20636F6D6520696D6D65AF
:10BFC00064696174656C790052656365697665645E
:10BFD00020424C455F47415454535F4556545F459A
:10BFE000584348414E47455F4D54555F5245515562
:10BFF0004553542028726571756573743A20256421
:10C000002C207265706C793A202564292E0000007E
:10C010002E2E5C2E2E5C2E2E5C2E2E5C2E2E5C6325
:10C020006F6D706F6E656E74735C6C696272617255
:10C030006965735C626F6F746C6F616465725C627A
:10C040006C655F6466755C6E72665F6466755F6280
:10C050006C652E6300000000436C69656E7420649B
:10C060006964206E6F74206861766520746865204D
:10C0700053657276696365204368616E6765642005
:10C08000696E6469636174696F6E2073657420748E
:10C090006F20656E61626C65642E4572726F723AD4
:10C0A00020307825303878006E72665F6673746F62
:10C0B000726167655F777269746528616464723D57
:10C0C00025702C207372633D25702C206C656E3DAD
:10C0D0002564206279746573292C207175657565F6
:10C0E0002075736167653A202564000043726561BD
:10C0F00074696E6720746865206F626A6563742076
:10C10000776974682073697A6520307825303878CB
:10C1100020776F756C64206F766572666C6F772020
:10C120006669726D776172652073697A652E204F3A
:10C1300066667365742069732030782530387820FE
:10C14000616E64206669726D776172652073697AC9
:10C1500065206973203078253038782E0000000083
:10C160002E2E5C2E2E5C2E2E5C2E2E5C2E2E5C63D4
:10C170006F6D706F6E656E74735C6C696272617204
:10C180006965735C626F6F746C6F616465725C6427
:10C1900066755C6E72665F6466755F7265715F6816
:10C1A000616E646C65722E63000000002E2E5C2EA2
:10C1B0002E5C2E2E5C2E2E5C2E2E5C636F6D706FAF
:10C1C0006E656E74735C6C69627261726965735CD2
:10C1D000626F6F746C6F616465725C6466755C6ECF
:10C1E00072665F6466755F7574696C732E630000B8
:10C1F0004D616A6F722053442075706461746520CC
:10C20000627574206E6F20424C2E2041626F7274F2
:10C2100020746F2061766F696420696E636170615C
:10C220006369746174696E672074686520424C2E7E
:10C230000000000054686520536F66744465766999
:10C2400063652073697A6520696E2074686520696A
:10C250006E666F2073747275637420697320746FD7
:10C260006F20736D616C6C20636F6D7061726564BB
:10C270002077697468207468652073697A65207214
:10C2800065706F7274656420696E207468652069DA
:10C290006E697420636F6D6D616E642E0000000026
:10C2A00054686520536F66744465766963652064DD
:10C2B0006F6573206E6F7420636F6E7461696E209A
:10C2C000746865206D61676963206E756D62657263
:10C2D000206964656E74696679696E672069742087
:10C2E0006173206120536F66744465766963652EBF
:10C2F00000000000496E76616C69646174696E6764
:10C3000020617070206265636175736520697420B7
:10C31000697320696E636F6D70617469626C65200A
:10C32000776974682074686520536F667444657615
:10C330006963652E000000002E2E5C2E2E5C2E2ED2
:10C340005C2E2E5C2E2E5C636F6D706F6E656E744E
:10C35000735C6C69627261726965735C626F6F7441
:10C360006C6F616465725C6466755C6E72665F6456
:10C3700066755F76616C69646174696F6E2E6300C7
:10C380002E2E5C2E2E5C2E2E5C2E2E5C2E2E5C63B2
:10C390006F6D706F6E656E74735C6C6962726172E2
:10C3A0006965735C626F6F746C6F616465725C6405
:10C3B00066755C6E72665F6466755F7665725F76E1
:10C3C000616C69646174696F6E2E63002E2E5C2E41
:10C3D0002E5C2E2E5C2E2E5C2E2E5C636F6D706F8D
:10C3E0006E656E74735C6C69627261726965735CB0
:10C3F00074696D65725C6578706572696D656E747F
:10C40000616C5C6170705F74696D6572322E63007F
:10C410002E2E5C2E2E5C2E2E5C2E2E5C2E2E5C6321
:10C420006F6D706F6E656E74735C6C696272617251
:10C430006965735C74696D65725C65787065726955
:10C440006D656E74616C5C6472765F7274632E638A
:10C45000000000002E2E5C2E2E5C2E2E5C2E2E5CFC
:10C460002E2E5C636F6D706F6E656E74735C6C699D
:10C47000627261726965735C6578706572696D6519
:10C480006E74616C5F6D656D6F626A5C6E72665F23
:10C490006D656D6F626A2E63000000002E2E5C2EAB
:10C4A0002E5C2E2E5C2E2E5C2E2E5C636F6D706FBC
:10C4B0006E656E74735C6C69627261726965735CDF
:10C4C0006578706572696D656E74616C5F736563C4
:10C4D00074696F6E5F766172735C6E72665F7365AE
:10C4E0006374696F6E5F697465722E63000000008B
:10C4F0004E52465F4552524F525F494E56414C494B
:10C50000445F4441544100004E52465F4552524FF1
:10C51000525F534F46544445564943455F4E4F542E
:10C520005F454E41424C4544000000004E52465F7C
:10C530004552524F525F464541545552455F4E4F0A
:10C54000545F454E41424C45440000004E52465F08
:10C550004552524F525F4D555445585F554E4C4FC2
:10C56000434B5F4641494C45440000004E52465FF4
:10C570004552524F525F4D555445585F4C4F434BB7
:10C580005F4641494C4544004E52465F4552524F2A
:10C59000525F4D555445585F434F4E445F494E4995
:10C5A000545F4641494C4544000000004E52465FEE
:10C5B0004552524F525F4D555445585F494E49546C
:10C5C0005F4641494C4544004E52465F4552524FEA
:10C5D000525F424C455F495053505F52585F504B39
:10C5E000545F5452554E4341544544004E52465FA9
:10C5F0004552524F525F424C455F495053505F5035
:10C600004545525F52454A454354454400000000A9
:10C610004E52465F4552524F525F424C455F495021
:10C6200053505F4C494E4B5F444953434F4E4E4528
:10C6300043544544000000004E52465F4552524F5D
:10C64000525F4150495F4E4F545F494D504C454DEC
:10C65000454E5445440000004E52465F4552524FED
:10C66000525F4E4F545F535550504F525445440003
:10C670004E52465F4552524F525F4D4F44554C45C6
:10C680005F4E4F545F494E495449414C495A4544C5
:10C69000000000004E52465F4552524F525F4D4FD0
:10C6A00044554C455F414C52454144595F494E49C0
:10C6B0005449414C495A4544000000004E52465FDF
:10C6C0004552524F525F4E4F545F464F554E4400B5
:10C6D0004E52465F4552524F525F494E56414C4969
:10C6E000445F5354415445004E52465F4552524FA9
:10C6F000525F444154415F53495A45004E52465F90
:10C700004552524F525F494F5F50454E44494E4744
:10C71000000000004E52465F4552524F525F535642
:10C72000435F48414E444C45525F4D495353494E37
:10C73000470000004E52465F4552524F525F494EED
:10C7400056414C49445F4C454E4754480000000058
:10C750004E52465F4552524F525F4452565F5457B5
:10C76000495F4552525F414E41434B004E52465F36
:10C770004552524F525F4452565F5457495F45529B
:10C78000525F444E41434B004E52465F4552524F1A
:10C79000525F494E5445524E414C00004E52465F46
:10C7A0004552524F525F53544F524147455F465591
:10C7B0004C4C00004E52465F4552524F525F4E5510
:10C7C0004C4C00004E52465F4552524F525F494E0C
:10C7D00056414C49445F504152414D004E52465FD4
:10C7E0004552524F525F4E4F5F4D454D0000000085
:10C7F0004E52465F4552524F525F464F5242494455
:10C8000044454E004E52465F4552524F525F44528D
:10C81000565F5457495F4552525F4F5645525255E5
:10C820004E0000004E52465F4552524F525F494EF5
:10C8300056414C49445F4144445200004E52465FC9
:10C840004552524F525F5245534F55524345530044
:10C850004E52465F4552524F525F494E56414C49E7
:10C86000445F464C414753004E52465F5355434345
:10C87000455353004E52465F4552524F525F424C11
:10C88000455F495053505F4348414E4E454C5F41D0
:10C890004C52454144595F45584953545300000098
:10C8A0004E52465F4552524F525F434F4E4E5F438A
:10C8B0004F554E54000000004E52465F4552524FB5
:10C8C000525F54494D454F55540000004E52465F4B
:10C8D0004552524F525F4255535900002E2E5C2E46
:10C8E0002E5C2E2E5C2E2E5C2E2E5C636F6D706F78
:10C8F0006E656E74735C6C69627261726965735C9B
:10C900006578706572696D656E74616C5F6C6F6778
:10C910005C7372635C6E72665F6C6F675F646566A2
:10C9200061756C745F6261636B656E64732E630026
:10C930002E2E5C2E2E5C2E2E5C2E2E5C2E2E5C63FC
:10C940006F6D706F6E656E74735C6C69627261722C
:10C950006965735C6578706572696D656E74616C2C
:10C960005F6C6F675C7372635C6E72665F6C6F673F
:10C970005F66726F6E74656E642E63007761726EAF
:10C98000696E670064656275670000001B5B313B80
:10C9900033306D001B5B306D000000001B5B313BD2
:10C9A00033316D001B5B313B33326D001B5B313B20
:10C9B00033336D001B5B313B33346D001B5B313B0C
:10C9C00033356D001B5B313B33366D001B5B313BF8
:10C9D00033376D00696E666F000000006572726F1C
:10C9E000720000002E2E5C2E2E5C2E2E5C2E2E5CF5
:10C9F0002E2E5C636F6D706F6E656E74735C6C6908
:10CA0000627261726965735C6578706572696D6583
:10CA10006E74616C5F73656374696F6E5F7661726B
:10CA2000735C6E72665F73656374696F6E5F697461
:10CA300065722E680000000073645F626C655F635E
:10CA400066675F73657428292072657475726E65F8
:10CA500064202573207768656E20617474656D703D
:10CA600074696E6720746F2073657420424C455F53
:10CA700047415454535F4346475F534552564943D9
:10CA8000455F4348414E4745442E000073645F6252
:10CA90006C655F6366675F736574282920726574CF
:10CAA00075726E6564202573207768656E206174E9
:10CAB00074656D7074696E6720746F20736574207F
:10CAC000424C455F434F4D4D4F4E5F4346475F5687
:10CAD000535F555549442E0073645F626C655F6314
:10CAE00066675F73657428292072657475726E6558
:10CAF00064202573207768656E20617474656D709D
:10CB000074696E6720746F2073657420424C455FB2
:10CB100047415454535F4346475F415454525F5416
:10CB200041425F53495A452E0000000073645F6222
:10CB30006C655F6366675F7365742829207265742E
:10CB400075726E6564202573207768656E20617448
:10CB500074656D7074696E6720746F2073657420DE
:10CB6000424C455F434F4E4E5F4346475F474150FF
:10CB70002E00000073645F626C655F6366675F73BD
:10CB8000657428292072657475726E65642025733A
:10CB9000207768656E20617474656D7074696E6766
:10CBA00020746F2073657420424C455F4741505F8D
:10CBB0004346475F524F4C455F434F554E542E00FE
:10CBC00073645F626C655F6366675F736574282971
:10CBD0002072657475726E656420257320776865B0
:10CBE0006E20617474656D7074696E6720746F2057
:10CBF00073657420424C455F434F4E4E5F4346473A
:10CC00005F474154542E00006170705F74696D6518
:10CC1000722E6D5F6466755F696E616374697669B3
:10CC200074795F74696D6572000000006170705FF7
:10CC300074696D65722E6D5F7764745F6665656497
:10CC40005F74696D657200006E72665F626F6F740B
:10CC50006C6F616465725F77647400006E72665F0A
:10CC60006466755F626C650062616C6C6F632E6DEB
:10CC70005F6275666665725F706F6F6C00000000C2
:10CC80006E72665F6466755F666C61736800000053
:10CC90006E72665F6466755F7265715F68616E640F
:10CCA0006C6572006E72665F6466755F736574743E
:10CCB000696E6773000000006E72665F6466755F80
:10CCC00073657474696E67735F73766369000000DF
:10CCD0006E72665F6466755F76616C6964617469C3
:10CCE0006F6E00006E72665F6466755F7665725F78
:10CCF00076616C69646174696F6E00006170705F69
:10CD000074696D657200000061746669666F2E6DEE
:10CD10005F7265715F6669666F0000006D656D5FCB
:10CD20006D6E6772000000006E72665F6673746FEE
:10CD3000726167650000000061746669666F2E6D40
:10CD40005F6669666F000000736F72746C6973745C
:10CD50000000000062616C6C6F632E6C6F675F6D2A
:10CD6000656D706F6F6C0000617070006E72665F51
:10CD7000736468006E72665F7364685F626C6500FE
:10CD80006E72665F7364685F736F63000200000019
:10CD900000000000F9290F00A5290F0067E6096AC5
:10CDA00085AE67BB72F36E3C3AF54FA57F520E51CC
:10CDB0008C68059BABD9831F19CDE05BFFFFFFFF9C
:10CDC000FFFFFFFFFFFFFFFF00000000000000006B
:10CDD0000000000001000000FFFFFFFFFCFFFFFF5D
:10CDE000FFFFFFFFFFFFFFFF00000000000000004B
:10CDF0000000000001000000FFFFFFFF512563FC61
:10CE0000C2CAB9F3849E17A7ADFAE6BCFFFFFFFFC5
:10CE1000FFFFFFFF00000000FFFFFFFF000000001A
:10CE200096C298D84539A1F4A033EB2D817D0377C4
:10CE3000F240A463E5E6BCF847422CE1F2D1176B5F
:10CE4000F551BF376840B6CBCE5E316B5733CE2B32
:10CE5000169E0F7C4AEBE78E9B7F1AFEE242E34F61
:10CE6000FFFFFFFF7F0000008000000000000000C7
:10CE700000000000FFFFFFFF7F00000080000000B7
:10CE80000000000000000000D4CF0F00B8570020C1
:10CE9000C40100006C150F0034D00F007C59002035
:10CEA000C46F00000E2E0F00A5440F00DD440F00DC
:10CEB0002D390F0051380F0008CC0F00000000037F
:10CEC0002CCC0F000000000348CC0F00000004042D
:10CED0005CCC0F000000040468CC0F0000000003CD
:10CEE00080CC0F000000040490CC0F00000004046C
:10CEF000A4CC0F0000000404B8CC0F000000040410
:10CF0000D0CC0F0000000404E4CC0F0000000404A7
:10CF1000FCCC0F000000000008CD0F000000000353
:10CF20001CCD0F000000000028CD0F0000000404FD
:10CF300038CD0F000000000348CD0F0000000000B6
:10CF400054CD0F000000000368CD0F000000040462
:10CF50006CCD0F000000030374CD0F00000003032D
:10CF600080CD0F000000030318580020106E002031
:10CF7000216E0020246E002034590020F4000000AF
:10CF8000C0580020B8580020C0580020D08700208A
:10CF90006859002018000000693A0F0000000000E6
:10CFA000397F0F0000000000717F0F0000000000BB
:10CFB000C58C0F0000000000518E0F000000000023
:10CFC000517F0F0000000000000000000200000080
:10CFD00071700F00011C1324590218200A15281C17
:10CFE00012FF031CFFFF0234011510014011021152
:10CFF000040A1954A0C1DA6028042520BD0F14DCEE
:10D00000C90F1A7C041AD4041A84041A94041A8CC2
:10D01000041A9C041AA4041AAC041AB4041ABC041A
:10D020001AC4041ACC04518490D0031BBD47143A8F
:04D0300010C50159CD
:020000041000EA
:0410140000100F00B9
:020000041000EA
:0410180000E00F00E5
:04000005000F1201D5
:00000001FF
